:020000040800F2
:10680000207C0020816A00089DBA000877A9000852
:1068100061B9000841730008E5D0000800000000DD
:10682000000000000000000000000000A169000856
:106830000775000800000000FD69000821C200087B
:106840009B6A00089B6A00089B6A00089B6A000814
:106850009B6A00089B6A00089B6A00089B6A000804
:106860009B6A00089B6A00089B6A00088174000804
:106870008D740008A1740008B5740008C174000884
:106880009B6A00089B6A00089B6A00089B6A0008D4
:106890009B6A00089B6A00089B6A00089B6A0008C4
:1068A0009B6A00089B6A0008DDC20008BDC20008A0
:1068B0009B6A000800000000000000009B6A0008BE
:1068C0009B6A00089B6A00089B6A00089B6A000894
:1068D0009B6A0008ADCE00089B6A00089B6A00080E
:1068E0009B6A00089B6A000800000000000000008E
:1068F0000000000000000000000000000000000098
:10690000000000009B6A0008000000009B6A00086D
:106910000000000000000000E9C200089B6A0008B7
:106920009B6A00089B6A00089B6A00089B6A000833
:106930009B6A00080000000000000000000000004A
:106940009B6A00089B6A00089B6A00080000000020
:106950009B6A00089B6A00089B6A00089B6A000803
:106960009B6A00089B6A00089B6A00080000000000
:106970009B6A00089B6A00080000000000000000FD
:106980009B6A00089B6A00089B6A0008DFF80CD02D
:1069900000F01EFB004800477DDD0008207C002041
:1069A0002C4B1968086800F05AB880F30988BFF3C7
:1069B0006F8F4FF0000080F31188704700000000D7
:1069C00008480068006880F308884FF0000080F3F2
:1069D000148862B661B6BFF34F8FBFF36F8F00DFCD
:1069E00000BF00BF08ED00E0DFF80C00016841F4D3
:1069F00070010160704700BF88ED00E0EFF309808F
:106A0000BFF36F8F134B1A681EF0100F08BF20EDF5
:106A1000108A20E9F04F106009B44FF0500080F365
:106A20001188BFF34F8FBFF36F8F08F053FB4FF008
:106A3000000080F3118809BC1968086800F014B8D8
:106A40001EF0100F08BF00F014B880F30988BFF3E0
:106A50006F8F7047A8010020EFF30580704730C8A2
:106A6000B0E8C04FFFF7A1BF30C8B0E8C04FFFF794
:106A7000E7BFB0EC088AB0EC08CAFFF7E6BF000039
:106A80000648804706480047FEE7FEE7FEE7FEE7C8
:106A9000FEE7FEE7FEE7FEE7FEE7FEE7ADC2000821
:106AA0008D6900082DE9F05F0546002092469B465F
:106AB00088460646814640241BE028464146474614
:106AC000224600F093F853465A46C01A914110D31B
:106AD00011461846224600F07AF82D1A67EB010895
:106AE0004F4622460120002100F071F817EB000903
:106AF0004E41201EA4F10104DFDC484631462A46FF
:106B0000434600F000B830BCBDE8C09F40EA010336
:106B10009B0703D009E008C9121F08C0042AFAD253
:106B200003E011F8013B00F8013B521EF9D2704717
:106B3000D2B201E000F8012B491EFBD270470022BF
:106B4000F6E710B513460A4604461946FFF7F0FF6C
:106B5000204610BD421C10F8011B0029FBD1801AF1
:106B6000704730B504460020034600E05B1C9342AA
:106B700003D2E05CCD5C401BF8D030BD00F0004299
:106B800030F000400AD0C10D01F56071C0F316006D
:106B900042EA0151C20840071143704700200146F4
:106BA000704730B50B46014600202022012409E041
:106BB00021FA02F59D4205D303FA02F5491B04FAB6
:106BC00002F52844151EA2F10102F1DC30BD202A95
:106BD00004DB203A00FA02F1002070479140C2F134
:106BE000200320FA03F3194390407047202A04DB66
:106BF000203A21FA02F00021704721FA02F3D04036
:106C0000C2F12002914008431946704710B5410077
:106C10000CD0C0F3C751962908DC7E2909DC06DBBD
:106C2000410204D000F0004040F07E5010BD002032
:106C300010BDC1F19604C4F1200100FA01F1E04059
:106C400000F0EAF9A04010BD2DE9FE4F804681EA30
:106C50000300C00F0C46009021F0004123F00045D6
:106C6000B8EB0200A94105D24046214690461C4699
:106C70000B46024623F00040104347D0270DC7F3D0
:106C80000A00C3F30A510290401A019040286BDABF
:106C9000C3F3130040F4801B0098924620B10023F8
:106CA000D2EB030A63EB0B0B01985946C0F140028B
:106CB0005046FFF78CFF06460D4650465946019A4E
:106CC00000F098F910EB08006141002487EA1152A6
:106CD00084EAE7731A4340D0009A62B3019A012A0A
:106CE0004FEA075215DC001B61EB02014FF0004236
:106CF00002EA0752CDE90042001C41F580113246FC
:106D00002B4600F0CFF903B000F045B840462146CD
:106D1000F9E7001B61EB0201001C41F5801300182C
:106D20005B412018A2F5001747EB030140EAD5703C
:106D3000B6196D4111E06D084FEA360645EAC07597
:106D40004FEA0752001B61EB0201001C41F5801164
:106D500049084FEA30000019514132462B4603B032
:106D600000F01CB800F08FB9009801224000002309
:106D7000D0EB020263EBE073009821464FEAE07427
:106D8000B8EB000061EB0401E9E783F000435BE747
:106D900081F0004158E730BCBDE8C08F30BCBDE891
:106DA000C04FFFF7DFBF2DE9FE4F81EA030404F077
:106DB000004421F0004100944FF0000B23F0004309
:106DC00050EA01045ED052EA03045BD0C3F30A54D4
:106DD000C1F30A552C44A4F2F3340194A0FB0254ED
:106DE000C1F3130141F48011C3F3130343F480137F
:106DF00001FB024400FB034E840A970A44EA8154D3
:106E000047EA8357A4FB076802958D0A05FB0785AF
:106E10004FEA932C04FB0C542705029D4FEA0658B9
:106E200047EA1637B5EB08056EEB070C870E920E96
:106E300047EA811742EA8312A7FB0201B6EB0B0176
:106E400064EB00042B0D43EA0C335E1844EB1C503A
:106E5000DA465146E7FB0201C5F313044FEA0B3350
:106E600043EA14534FEA0432019C43EA0603A4F1B7
:106E70000C040294009CCDE900B400F013F903B0B7
:106E800000F003B800200146F9E730BCBDE8C08F30
:106E90002DE9F04D81EA030404F0004B21F0004598
:106EA00014464FF0000A23F0004150EA050220D0BA
:106EB00054EA01021DD0C5F30A570246C5F3130375
:106EC000C1F31300C1F30A5640F4801543F4801354
:106ED000A7EB0608101BD64608F2FD3873EB050039
:106EE00002D308F1010801E092185B41B8F1000FEC
:106EF00003DA00200146BDE8F08D00204FF4801138
:106F0000064684460EE0171B73EB050705D3121BDC
:106F100063EB050306434CEA010C49084FEA3000D5
:106F200092185B4150EA0107EDD152EA030012D0FA
:106F300082EA040083EA0501084305D0101BAB4137
:106F400006D20122002306E000224FF0004302E0B7
:106F50006FF0010253101AEB06004CEB085110EBD6
:106F60000A0041EB0B01BDE8F04D00F08CB8C1F315
:106F70000A52C1F3130140F2FF3341F480119A42E7
:106F800002DA00200146704740F233439A42A2F2EF
:106F9000334202DC5242FFF729BEFFF718BE000061
:106FA00030B5041E71F1000404DB4FF00044404290
:106FB00064EB0101141E73F1000405DB1C464FF065
:106FC0000043524263EB0403994208BF904230BD34
:106FD000064C074D06E0E06840F0010394E8070026
:106FE00098471034AC42F6D3FFF7D4FCC8FD000834
:106FF000E8FD0008202A06DBCB17203A41FA02F010
:1070000043EAE07306E041FA02F3D040C2F1200205
:1070100091400843194670470029A8BF7047401C9B
:10702000490008BF20F00100704710B4B0FA80FC9E
:1070300000FA0CF050EA010404BF10BC704749B1DB
:10704000CCF1200421FA04F411FA0CF118BF01214B
:1070500021430843A3EB0C01CB1D4FEA00614FEA2B
:10706000102042BF002010BC704700EBC3501044FA
:107070000029A4BF10BC7047401C490008BF20F085
:10708000010010BC704710B5141E73F1000408DA3B
:10709000401C41F1000192185B411A4301D120F0DC
:1070A000010010BD2DE9F04D92469B4611B1B1FA99
:1070B00081F202E0B0FA80F220329046FFF787FDBD
:1070C00004460F4640EA0A0041EA0B0153465A467D
:1070D000084313D0114653EA010019D0C8F1400209
:1070E0005046FFF783FD05460E4650465946424638
:1070F000FFF76DFD084305D0012004E02046394626
:10710000BDE8F08D0020054346EAE0762C43374386
:107110000A986305E40AA0EB08000022FD0A44EA8D
:1071200047540A3002D500200146E9E7010510194D
:107130006941DDE9084500196941BDE8F04DA2E764
:1071400070B58C1810F8015B15F0070301D110F829
:10715000013B2A1106D110F8012B03E010F8016B56
:1071600001F8016B5B1EF9D12B0705D40023521ED9
:107170000DD401F8013BFAE710F8013BCB1A921C41
:1071800003E013F8015B01F8015B521EF9D5A1423F
:10719000D8D3002070BD10B5846A616D11F0500F16
:1071A00006D0616DC90625D5204600F06EFD10BDE4
:1071B000606D40F40070606520680168090716D5AD
:1071C00003F061FC78B12068C068800400280ADB05
:1071D000606D20F480706065606DC00403D4606DE4
:1071E00040F001006065204600F04DFD10BDC06814
:1071F0008007EBE7E16C496BBDE81040084710B52C
:10720000806A416D41F040014165816D41F00401AA
:10721000816500F03AFD10BD10B5806A00F034FDC4
:1072200010BD000070B50446006881688268C1F333
:10723000400112F0010F28D039BB816801F00D0127
:10724000012914D18168124A1140891C816021688A
:107250000320086001F0C8FA054612E001F0C4FA04
:10726000401B02280DD920688068C00709D0606DD6
:1072700040F010006065A06D40F00100A0650120A5
:1072800070BD20688068C007E8D1002070BD000094
:10729000C0FFFF7FF8B50446002000902068816899
:1072A00011F0010F41D18168214A11422ED181682C
:1072B000D5432940491C81601E48806800F0E07079
:1072C00000020DD51C481D490068B0FBF1F0401CC0
:1072D00000EB4000800000E0401E00900028FBD141
:1072E00001F082FA06461BE0816811F0010F03D11C
:1072F00081682940491C816001F076FA801B0228D0
:107300000ED920680068C043C00709D0606D40F006
:1073100010006065A06D40F00100A0650120F8BD7F
:1073200020680168C943C907DED10020F8BD00000C
:107330003F0000800003045074000020400D030053
:10734000FEE700001FB5DFF89C90DFF89CA0DFF897
:107350009CB0DFF89C8000BF99ED000A8AED000A1E
:1073600099ED030A8BED000AD8F80C00FFF706FC34
:1073700006460F46D8F81000FFF700FC04461D48EB
:107380000D460068FFF7FAFB8DE8F00041EC100BAA
:1073900019A053EC102B05F0A7FEC82006F026FD1F
:1073A00098F8000010B922A005F09EFE98F80000A1
:1073B0004446012802D122A005F096FE207802283A
:1073C00002D123A005F090FE2078032802D124A04A
:1073D00005F08AFE20780428BED125A005F084FEA1
:1073E000BAE70000881B00201C01002020010020BB
:1073F00000000020800000206375725F616E676C82
:10740000655F6465673D5B252E32665D204D6F7458
:107410006F725F7370655B252E32665D204D6F74F1
:107420006F725F6375725B252E33665D0D0A000017
:10743000436C6F7365206F7574707574200D0A004E
:10744000436C6F736520696E707574200D0A0000BF
:107450004F70656E3120696E707574200D0A0000E2
:107460004F70656E3220696E707574200D0A0000D1
:1074700064656661756C745F48616C6C200D0A0010
:10748000014800F045BE00001016002010B503486A
:1074900000F03EFEBDE8104004F07ABBDC1700208F
:1074A00010B5034800F034FEBDE8104004F070BB96
:1074B00024180020014800F02BBE0000BC19002059
:1074C000014800F025BE00007419002030B590F886
:1074D000444004F01C050124AC40056C6C60046859
:1074E00063608368102B036803D099600068C260F2
:1074F00030BD9A600068C16030BD04F01DFC1420EE
:1075000006F074FCF9E7704770B500231C4611E0E3
:1075100011F82350055531F823502E0A05196E70C5
:1075200051F82360360CAE7051F823605B1C360EA8
:10753000EE70241D9442EBD370BD72B6FEE70000DE
:10754000144A117F1448012901D003290FD103687F
:1075500023F400730360036843F40063036003686B
:1075600023F400630360036843F40073036002299B
:1075700001D003290BD1016841F4805101600168F9
:1075800021F480510160016841F4806101600020B4
:10759000107770475400002000200240C1070548C2
:1075A00003D0416941F004014161416941F48031F6
:1075B000416170470020024008494A69C0B222F484
:1075C0007E7242EAC0004861486940F002004861AA
:1075D000486940F480304861704700000020024054
:1075E000054910B54C6944F001044C610260BFF3D9
:1075F0006F8F436010BD000000200240094A10B5A3
:107600005469402344F480245461EFF3108272B62D
:1076100010C910C05B1E13F0FF03F9D182F310886C
:1076200010BD00000020024070B5054601F0DCF8F6
:107630000646134C08E0681C06D001F0D5F8801B04
:10764000A84201D3032070BD2069C003F3D4206990
:107650000C4908400CD00C494A6802434A60810F2B
:1076600001D0A169A161810000D02061012070BD1D
:107670002069C00701D001202061002070BD0000FA
:1076800000200240FAC302005400002070B586B00A
:107690000C00054628D01548854225D800260496BA
:1076A00000F0FCFE1248816941F0404181614CF2DA
:1076B000FA3101612846009600F01CF80190284636
:1076C00000F026F8029005EB8400401E00F020F840
:1076D0000299401A401C039004A9684600F00EFE6F
:1076E000002801D000F07AFE06B070BD000004084A
:1076F000002002400449096804494FF0010009686C
:10770000CA431204120C704700000140E075FF1FCD
:107710000E4910B509684FF48024CB431A04120CAB
:107720000AD00A045FEA921202F10062824205D98D
:10773000A0F10060C00A10BD2246F5E71A04120C41
:1077400001D009048C09001BF2E70000E075FF1F5F
:10775000084B10B598420CD883070AD1D21C930865
:10776000002204E050F8224041F82240521C9A4284
:10777000F8D310BD000004082DE9F04117460D466E
:10778000044600F08BFE0F48844216D2002609E022
:10779000D5E900232146002000F02AFE68B908340C
:1077A0000835761CB6EB570FF2D3F80705D063689F
:1077B000214600202A6800F01BFEBDE8F04100F0E1
:1077C0000DBE0000000004082DE9F04117460E46EA
:1077D000044600F063FE0A4884420DD2002509E009
:1077E000D6E900232146002000F002FE20B908342B
:1077F0006D1C0836BD42F3D3BDE8F04100F0EEBD8C
:1078000000000408F8B500260446009690F85000E1
:107810000D4601280BD0012084F850002046FFF7C8
:1078200001FD0100606D04D040F010002BE002204B
:10783000F8BD20F4885040F002006065206882683E
:10784000134B1A4005F080431A4342F00042826015
:107850004FF4912320680EE0009A521C00929A4245
:1078600009D3606D20F0020040F01000606584F8DC
:1078700050600120F8BD8268D20FEDD1606D20F01C
:10788000020040F00100606584F850600846F8BDD1
:10789000C0FFFF3F2DE9F84F00270446009790F8FE
:1078A0005000DFF8B0930D46B846012811D00126EC
:1078B00084F85060206803F0E2F860B1606D40F039
:1078C000200060655FF0010784F85080384600F0C2
:1078D000D7B90220FBE769680C20052912D80229D4
:1078E00007D0032907D0042907D0052907D006218E
:1078F00007E0686006E0122103E0182101E04FF480
:1079000080716960D5E90021236800EA911018446C
:10791000036B01F01F014FF01F0C0CFA01FCC2F3C6
:10792000846223EA0C038A4013430363206803F054
:10793000A6F88246206803F09EF85AEA00001DD19E
:10794000AA682968206803F0A6F820686969C268F7
:10795000C2F3C102520091402A69042A0FD000EB01
:1079600082002B68026EDFF8F0C203F0F84302EAEF
:107970000C020B431A4342F00041016672E0002101
:1079800003F073F8400320684FF0000172D003F059
:107990006CF890FAA0F0B0FA80F1286842036ED03B
:1079A00090FAA0F0B0FA80F0814204D10022114692
:1079B000206803F07FF80121206803F056F84003A7
:1079C00020684FF001015DD003F04FF890FAA0F06D
:1079D000B0FA80F12868420359D090FAA0F0B0FACA
:1079E00080F0814204D100220121206803F062F876
:1079F0000221206803F039F8400320684FF00201AB
:107A000048D003F032F890FAA0F0B0FA80F128687C
:107A1000420344D090FAA0F0B0FA80F0814204D141
:107A200000220221206803F045F80321206803F0BA
:107A30001CF8400320684FF0030133D003F015F821
:107A400090FAA0F0B0FA80F1286842032FD090FAA3
:107A5000A0F0B0FA80F0814204D100220321206816
:107A600003F028F82068816811F0010F22D0ABE004
:107A700000E004E002F0F9FFC0F384618DE7C0F399
:107A8000846091E702F0F1FFC0F38461A2E7C0F3E4
:107A90008460A6E702F0E9FFC0F38461B7E7C0F3B2
:107AA0008460BBE702F0E1FFC0F38461CCE7C0F380
:107AB0008460D0E72A7B296850F8B03FC1F3120CEC
:107AC00023EA0C0302F0180C644A22FA0CF20A4072
:107AD00013430360E968494576D1286841031BD008
:107AE00090FAA0F1B1FA81F1491C01F01F010929B6
:107AF0004FEA403131D8002911D090FAA0F1B1FA03
:107B000081F100BF01F1010101F01F0106FA01F648
:107B100008D1C0F3846109E0C0F38461E4E7C0F3F5
:107B20008461EFE790FAA0F1B1FA81F101F101016E
:107B300001F01F0146EA816102D1C0F3846003E0D5
:107B400090FAA0F0B0FA80F000F1010000F01F0000
:107B500000EB400041EA005132E000290ED090FADB
:107B6000A0F1B1FA81F100BF01F1010101F01F01A3
:107B700006FA01F605D1C0F3846106E0C0F3846122
:107B8000F2E790FAA0F1B1FA81F101F1010101F0FF
:107B90001F0146EA816102D1C0F3846003E090FADC
:107BA000A0F0B0FA80F000F1010000F01F002C4AB4
:107BB00000EB400002EB005041EA000141F000718F
:107BC000AA68206802F067FF26482A6802423FF44C
:107BD0007BAE25488168254D254B01F0E071AA4216
:107BE0001BD10D0219D422689A427FF46DAE8268CF
:107BF00041F4000122F0E0720A4382601D481E49F0
:107C00000068B0FBF1F0401C00EB4000800000E099
:107C1000401E00900028FBD156E6184DAA4207D11D
:107C2000CD0105D422689A42F6D141F080710AE074
:107C30006FF00045EA42EFD14A02EDD422689A4241
:107C4000EAD141F48001826822F0E0720A43826046
:107C50003AE6000000007F4000F0FF03FFFF07004E
:107C6000000020FE0000088000030450000052C7FE
:107C70000000045074000020400D0300000084CB7D
:107C800018BCBDE8E08F704770477047F8B54FF0FB
:107C9000000504002E46009502D0606D10B107E08B
:107CA0000120F8BD204600F0C9F8A66584F85060B0
:107CB00020688168C1F3407119B18168574A114049
:107CC000816020688168C1F3007189B98168544A74
:107CD000114041F080518160524853490068B0FB27
:107CE000F1F04000801C00E0401E00900028FBD115
:107CF00020688168C1F3007141B9616D41F01001E4
:107D00006165A16D41F00101A165012502F0B7FE99
:107D1000616D01F010010143606D05D040F010006D
:107D2000606501252846F8BD20F4807040F002000F
:107D300060652068806810F0010F0BD13B488068B7
:107D400010F0010F06D13A486168826822F47C1273
:107D50000A438260E168606B627E0843A16841EA81
:107D60004231084394F8201040EA0140012904D12F
:107D7000A18C304A02EB41410843A16A29B101F4C8
:107D80007071E26A014342EA01002268D1682A4B1D
:107D900019400143D160206802F071FE0646206858
:107DA00002F069FE304315D1207E94F83010800334
:107DB00040EA41022068C16844F20203994311433A
:107DC000C16094F8380001280CD02068016921F0C6
:107DD00001010161206901282068016B21F00F0178
:107DE00011D013E0D4E90F010843D4E91112114373
:107DF000084321680A6940F2FC739A43104340F03B
:107E000001000861E6E7E269521E11430163606DFB
:107E100020F0020040F00100606583E7C0FFFF5FD3
:107E2000C0FFFF7F74000020400D030000000450DD
:107E3000000304500000FEFF07C0F0FFF0B59DB046
:107E40000646142117A8FEF77AFE5C216846FEF765
:107E500076FE2F493068884258D14FF48040009018
:107E60008003149002240120CDE9014008200390F2
:107E70000720CDE904048801CDE90640684600F0FA
:107E8000B3FE08B1FFF759FB2249C86C40F400501B
:107E9000C864C86C00F400501C90C86C40F001002D
:107EA000C864C86C00F001001C90C86C40F002006F
:107EB000C864C86C002500F002001C90F0200B275D
:107EC0001995CDE9170717A94FF0904000F09CFBDA
:107ED0001995CDE9174717A90F4800F095FB104CED
:107EE0000E48C4E900058020A560C4E903504000A5
:107EF00060618000A0612020C4E90705204600F0F1
:107F000065F908B1FFF719FBF464A6621DB0F0BD76
:107F10000000045000100240000400480800024025
:107F20001016002070B5044615460E46006802F093
:107F3000A6FDE0BB94F85000012842D0012084F84F
:107F400050002046FFF7A6F9002110B184F8501028
:107F500070BD606D40F60162904340F480706065D2
:107F6000606DC00404D5A06D20F00600A06500E09F
:107F7000A165E26C1448D062E26C14481063E26CB4
:107F80001348506322681C20106084F85010206849
:107F9000416841F0100141602068C16841F0010171
:107FA000C16021682B4632464031E06C00E008E0B9
:107FB00000F06CF921688A68064B1A40121D8A602D
:107FC00070BD022070BD0000977100081972000892
:107FD000FF710008C0FFFF7F10B590F82510002248
:107FE000022905D00421C16380F82420012010BD9E
:107FF00001680B6823F00E030B6001680B6823F027
:1080000001030B6090F84410046C01F01C03012183
:1080100001FA03F3636080F8251080F824201046ED
:1080200010BD10B590F825100024022903D00421BA
:10803000C16301241AE001680A6822F00E020A6096
:1080400001680A6822F001020A6090F84410036C8B
:1080500001F01C02012101FA02F25A6080F8251099
:10806000002180F82410816B01B18847204610BDA3
:1080700030B590B101680A6822F001020A60204C14
:10808000036814211F4AA34209D21F4C1C44B4FBAD
:10809000F1F18900C0E910210BE0012030BD184C3E
:1080A00064421C44B4FBF1F189004164144908396D
:1080B00001640021196090F8443003F01C0401238E
:1080C000A340046C6360046C0F23944202D152F805
:1080D000A84F02E00A4AA032146890F8445005F014
:1080E0001C05AB409C431460C16201634163816322
:1080F000C16380F8251080F82410002030BD0000F6
:108100000804024000000240F8FFFDBFC06B70474A
:10811000F0B4016C0C6801680D6890F8442002F01E
:108120001C06042202FA06F3234211D06B070FD576
:108130000B689B0603D40B6823F004030B6090F8D4
:10814000441001F01C018A40016C4A60016B1DE083
:10815000022303FA06F727424FF0000C4FF001020A
:1081600018D0AF0716D50C68A40605D40C6824F007
:108170000A040C6080F8252090F8441001F01C01DE
:108180008B40016C4B6080F824C0C16A00291AD072
:10819000F0BC08470823B340234214D02B0712D564
:1081A0000B6823F00E030B6090F84410036C01F091
:1081B0001C0102FA01F15960C26380F8252080F8A1
:1081C00024C0416BE2E7F0BC7047000070B568B1B5
:1081D0002B4C036814212B4AA34209D22A4C1C447D
:1081E000B4FBF1F18900C0E910210BE0012070BD62
:1081F000234C64421C44B4FBF1F1890041642049E2
:1082000008390164022180F825101C6847F6F071D6
:108210008C43D0E902152943D0E90456354329435C
:1082200085692943C5692943056A294321431960A2
:108230008168B1F5804F19D0036C0F21934202D1B0
:1082400052F8A83F02E00E4AA032136890F844406A
:1082500004F01C04A1408B43136090F84430416843
:1082600003F01C0399401368194311600021C16396
:10827000012280F8252080F82410084670BD0000F7
:108280000804024000000240F8FFFDBF70B504463C
:1082900090F82400002501280CD0012084F8240047
:1082A00094F825600020012E06D084F824000225D1
:1082B000284670BD022070BD022684F82560E06368
:1082C0002068066826F0010606602046FFF7FEF8E3
:1082D000206B00282068016802D041F00E0106E002
:1082E00021F0040101602068016841F00A01016089
:1082F0002068016841F001010160D9E72DE9F05FD4
:10830000054632488946017801290CD0012680466D
:1083100006704CF2503B5846FFF786F907004FF0C5
:10832000000A03D04EE0022000F054B85146404607
:10833000C8F804A0264C226892050AD52168490590
:1083400005D5216821F480612160032109E00677C9
:1083500008E02268520504D5216821F4806121607B
:10836000022101772868012807D04FF0FF31C9F8B2
:10837000001040F2FA3BAE681DE06868FFF70EF9A6
:108380005846FFF751F90746606920F00400606124
:1083900016E030466968FFF70FF94CF25030FFF7EE
:1083A00043F90700606920EA0B00606102D0C9F858
:1083B000006005E0761CD5E902010844B042E8D827
:1083C000FFF7BEF888F800A03846ADE7540000205B
:1083D0000020024030BCBDE8C09F00000348416956
:1083E00041F0004141610020704700000020024040
:1083F0002DE9FF5F254C0646904620789A460128D5
:108400000BD0012020704CF2503B5846FFF70CF97E
:1084100007004FF0000904D02AE0022004B000F069
:1084200039B84846C4F80490194D2968490504D55F
:10843000286820F4806028600220207726B1012E71
:1084400009D0022E07D00CE0424653460198FFF7B0
:10845000C7F8012612E041460198FFF7CFF8022E37
:108460000AD05846FFF7E0F84FEA0007FFF768F830
:1084700084F800903846D1E74FF480265846FFF73D
:10848000D3F807466869B0436861EFE754000020FD
:108490000020024030BCBDE8C09F0000064900201B
:1084A0004A69002A07DA054A8A60054A8A604969EA
:1084B000002900DA012070470020024023016745AF
:1084C000AB89EFCD2DE9F84F00230126DFF818C165
:1084D0000F2782E006FA03F414EA01027CD023F0AD
:1084E00003056544AA46D5F808909D074FEA157E16
:1084F00007FA0EF505EA090B0095B0F1904F05D08B
:108500003A4DA84205D14FF0010816E04FF000089F
:1085100013E0374DA84202D14FF002080DE0354D6F
:10852000A84202D14FF0030807E0334DA84202D120
:108530004FF0040801E04FF0070808FA0EF8D8459C
:1085400026D1DFF8B880D8F8009029EA0209C8F8E7
:10855000009008F10408D8F8009029EA0209C8F848
:108560000090DFF8988008F10C08D8F8009029EA0C
:108570000209C8F80090A8F10408D8F80050954303
:10858000C8F80050009DDAF80820AA43CAF808206D
:10859000D0F800804FEA4309032202FA09F248EAC0
:1085A0000208C0F80080DD0800EB8505AA46D5F872
:1085B00020804FEA43794FEAD96907FA09F528EA9A
:1085C0000508CAF820808568954385604568A543FD
:1085D0004560C4689443C4605B1C31FA03F27FF4C5
:1085E00079AF00F00DB80000000001400004004821
:1085F00000080048000C004800100048000401403A
:1086000018BCBDE8E08F00002DE9F04FDFF8AC9119
:1086100000230325A9F1040B85B04FF0010C0F27AF
:1086200009F1040AABF1040EBFE000BF0CFA03F637
:10863000324075D00C7904F00304012C01D0022CD7
:108640001BD1846800945C0005FA04F80494009C33
:1086500024EA08040094D1F80C80049C08FA04F879
:10866000009C48EA0408C0F808804468B4430E79C6
:10867000C6F300169E40264346600C79E443A407E7
:108680000AD0C4684FEA430805FA08F6B4438E6876
:1086900006FA08F62643C6600C7904F00304022C9F
:1086A00010D1DC0800EB84040294246A5E074FEAD0
:1086B000D66807FA08F6B4430E6906FA08F62643A8
:1086C000029C266204684FEA430805FA08F6B443A0
:1086D0000E7906F0030606FA08F6264306604C6893
:1086E00014F4403F60D0364C266E46F001062666F4
:1086F000246E23F0030604F001040094314C34444A
:108700000294A4689E074FEA167807FA08F6B44365
:10871000B0F1904F05D02C4EB04204D1012612E0AA
:1087200042E000260FE0294EB04201D102260AE0C5
:10873000274EB04201D1032605E0264EB04201D1BA
:10874000042600E0072606FA08F62643029CA660E7
:10875000D9F800604C46D1F8048096435FEAC828F7
:1087600000D516432660DAF800405646D1F804805A
:1087700094435FEA882800D514433460DBF8004056
:108780005E46D1F8048094435FEA883800D51443EC
:108790003460DEF800407646D1F8048094435FEA06
:1087A000C83800D5144334605B1C0A6832FA03F4FD
:1087B0007FF43CAF05B000F00FB8000008040140A2
:1087C000001002400000014000040048000800487A
:1087D000000C00480010004830BCBDE8C08F0AB152
:1087E000816170478162704701488068704700006E
:1087F0004800002090F84120202A24D190F8402001
:10880000012A20D0012280F84020242280F8412033
:108810000268136823F0010313600268136823F4ED
:1088200080531360026813680B43136001680A6881
:1088300042F001020A60202180F84110002180F8F6
:108840004010084670470220704790F84120202AC7
:1088500022D190F84020012A1ED0012280F8402029
:10886000242280F841200268136823F0010313607A
:108870000268136823F4706343EA01211160016800
:108880000A6842F001020A60202180F841100021AC
:1088900080F84010084670470220704770B5040009
:1088A00004D094F84100002510B106E0012070BD0D
:1088B00084F84050204600F04DF8242084F8410010
:1088C0002068016821F0010101606068216820F0E2
:1088D000706008612068816821F400418160E0686F
:1088E0000128A06807D040F4044021688860E0684F
:1088F000022803D006E040F40040F6E721684FF478
:108900000060486020684168114A11434160206856
:10891000C16821F40041C160D4E904010843A169A0
:1089200040EA01202168C860D4E9070108432168B2
:1089300008602068016841F0010101606564202041
:1089400084F84100256384F84250002070BD000087
:108950000080000230B59DB00446142117A8FEF730
:10896000EEF85C216846FEF7EAF81749206888426D
:1089700027D18020002500900D95684600F034F93D
:1089800008B1FEF7DAFD114CE06C40F00200E06443
:10899000E06C17A900F002001C904FF4C040179043
:1089A0001220CDE918050420CDE91A500848FFF738
:1089B0002BFEA06D40F48000A065A06D00F4800047
:1089C0001C901DB030BD0000005800400010024057
:1089D00000040048024881680278114481607047B1
:1089E0004800002010B50024032000F0AFF80F204D
:1089F00000F008F808B1012401E000F04FF820462B
:108A000010BD000030B505461F4887B0816D41F0AC
:108A100010018165806D06A900F01000009001A88A
:108A200000F0E2FA0498B0B100F0FEFA40001749F5
:108A3000174AB0FBF1F11748491E0260416040F24D
:108A4000E7320021C0E903218160816100F04CFE22
:108A5000040003D015E000F0E7FAE8E70D4800F065
:108A600019FF04000DD1362000F043F8102D07D275
:108A700000222946362000F049F80748056000E04A
:108A8000012407B0204630BD0010024040420F00D4
:108A900000100040301B00204C0000200B4882B02A
:108AA000016E41F001010166016E01F001010091CA
:108AB000816D41F080518165806D002200F0805011
:108AC00000900F21901E02B000F020B8001002406C
:108AD00000280DDB00F01F020121914040098000B9
:108AE00000F1E020C0F88011BFF34F8FBFF36F8F0C
:108AF0007047002809DB00F01F0201219140400966
:108B0000800000F1E020C0F800117047F0B40E4B77
:108B10001B680C46C3F30223C3F10705042D00D9DB
:108B20000425191D072901D2002300E0DB1E0126C0
:108B300006FA05F1491E214099409E40761E1640D6
:108B40003143F0BC04F0E0BA0CED00E0064900F05F
:108B5000070208684FF6FF03184040EA0220034A64
:108B600010430860704700000CED00E00000FA05BB
:108B70001649B0F5007F0868C0F3412009D00228EB
:108B800005D0086820F4C06040F4806008600020D0
:108B900070470128FBD0086820F4C06040F40070E2
:108BA00008600B483222006850430A4AB0FBF2F0DA
:108BB000401C00E0401E4A69520501D50028F9D149
:108BC00048694005E3D5032070470000007000406D
:108BD0007400002040420F000248006800F4C060AA
:108BE00070470000007000402DE9F84F0446002750
:108BF0000088A84D3E46000515D5606C60B1B0F503
:108C0000000F04D0B0F5400F2BD001270AE0E86830
:108C100040F48030E86024E00021201D03F0B8F823
:108C200007001ED03E46206880033AD5A86D4FF05D
:108C30000008C00009D4A86D40F08050A865A86D58
:108C40004FF0010800F080500090DFF84CA2DAF8F5
:108C5000001041F48071CAF80010FFF7C5FD81468D
:108C600010E0D5F88800616C20F440000843C5F896
:108C70008800D8E7FFF7B8FDA0EB0900022801D96A
:108C8000032705E0DAF80000C005F3D5002F7DD0FA
:108C90004FEA0706B8F1000F03D0A86D20F080500E
:108CA000A8652078C00707D0D5F88800216A20F091
:108CB00003000843C5F888002078800707D5D5F859
:108CC0008800616A20F00C000843C5F8880020780D
:108CD000400707D5D5F88800A16A20F03000084386
:108CE000C5F888002078800607D5D5F88800E16AA5
:108CF00020F440600843C5F888002088800507D527
:108D0000D5F88800E16B20F440200843C5F88800BE
:108D10002088400507D5D5F88800216C20F4401044
:108D20000843C5F888002078400607D5D5F88800A4
:108D3000216B20F440500843C5F8880020780006D5
:108D400007D5D5F88800616B20F440400843C5F88A
:108D500088002088C00507D5D5F88800A16B20F4CD
:108D600040300843C5F8880020684FF000670003D2
:108D70004FF0806850D5D5F88800A16C20F0406095
:108D80000843C5F88800A06CB84200E005E03BD17C
:108D9000E86840F48010E8603EE0D5F8900010F4F8
:108DA000407014D0A16D814211D0D5F89000D5F853
:108DB000901020F4407041F48031C5F89010D5F83F
:108DC000901021F48031C5F89010C5F89000C007CC
:108DD00011D0FFF709FD074641F2883907E000BFCF
:108DE000FFF702FDC11B494501D9032652E7D5F81B
:108DF00090008007F4D5D5F89000A16D20F4407064
:108E00000843C5F8900045E7404505D10121201DE4
:108E100002F0BEFF00B106462068400317D5D5F822
:108E20008800E16C20F040600843C5F88800E06CE1
:108E3000B84204D1E86840F48010E86007E040459B
:108E400005D10121201D02F0A3FF00B106462088B4
:108E5000400411D5D5F88800216D20F0405008431A
:108E6000C5F88800206DB0F1805F05D10221201D7A
:108E700002F08EFF00B106462088000406D555F8A2
:108E8000880F616D20F0804008432860304600F074
:108E900005B80000001002400070004018BCBDE89A
:108EA000E08F00002DE9F0470F4605006BD0494EDA
:108EB000306800F00700B84209D2306820F007009F
:108EC00038433060306800F00700B8425BD1287842
:108ED000414C80070AD5A868A16801F0F0018842DA
:108EE00004D9A16821F0F0010143A1602878C007EE
:108EF0002CD06868032811D0022812D0216898B1BC
:108F0000490500293FDAA16821F003010143A1606E
:108F1000FFF76AFC804641F2883910E02168890138
:108F2000EFE721688903ECE78907EAE7FFF75CFCD4
:108F3000A0EB0801494502D90320BDE8F087A068ED
:108F4000696800F00C00B0EB810FEFD12878800742
:108F50000AD5A868A16801F0F001884204D2A1688E
:108F600021F0F0010143A160306800F00700B84231
:108F70000BD9306820F0070038433060306800F0CB
:108F80000700B84201D00120D7E72878400705D56F
:108F9000A068E96820F4E0600843A0602878000732
:108FA00006D5A068296920F4605040EAC100A0609D
:108FB00000F05EF8A168094AC1F30311515C01F0A9
:108FC0001F01C8400649086006480068BDE8F04730
:108FD000FFF718BD0020024000100240E0FC00082E
:108FE000740000204C0000200F2202600C4A93689D
:108FF00003F003034360936803F0F0038360936816
:1090000003F4E063C36092684FF4E06303EAD202C2
:1090100002610448006800F0070008607047000023
:109020000010024000200240054806490068896897
:10903000054AC1F30221515C01F01F01C84070478D
:10904000740000200010024020FD00080548064979
:1090500000688968054AC1F3C221515C01F01F0113
:10906000C8407047740000200010024020FD000836
:1090700070B52549002318468A68CC6812F00C02A6
:1090800004F00306214C4FEA640509D00C2A05D0F0
:10909000042A32D0082A00D1284670BD012E10D1F2
:1090A0000B681B0704D4D1F89430C3F3032302E008
:1090B0000B68C3F30313164E56F82330DAB10C2AAB
:1090C000EBD1C86800F00300022818D0032818D09C
:1090D0001846CA68CB68C2F30212C3F3062343439F
:1090E000521CB3FBF2F2C868C0F34160401C400060
:1090F000B2FBF0F070BD184670BD204670BD204632
:10910000E7E72846E5E70000001002400024F400ED
:10911000F0FC00082DE9F84304006FD0FA4DA86870
:1091200000F00C06E86800F003072078C00664D55C
:1091300076B10C2E01D1012F0AD0A0690028286831
:109140007AD040F001002860FFF74EFB80465DE0DA
:109150002868800702D5A0690028DED0216A286827
:10916000000703D5286800F0F00004E0D5F894006B
:10917000F02202EA1010814216D9084602F09EFE43
:1091800000283BD1286840F0080028602868216A40
:1091900020F0F000084328606868E16920F47F400F
:1091A00040EA0120686016E0286840F00800286066
:1091B0002868216A20F0F000084328606868E169A7
:1091C00020F47F4040EA0120686026B9206A02F05E
:1091D00075FE0028D5D1FFF74BFFA968CB4AC1F334
:1091E0000311515C01F01F01C840C9490860C9481A
:1091F0000068FFF707FC00287ED12EE0CAE000BF20
:10920000FFF7F2FAA0EB0800022876D8286880075A
:10921000F6D5286840F0080028602868216A20F008
:10922000F000084328606868E16920F47F4040EA64
:109230000120686011E0FFE720F001002860FFF7DF
:10924000D3FA804606E000BFFFF7CEFAA0EB080095
:109250000228DAD828688007F6D42078C00740D0E2
:10926000082E18D00C2E01D1032F14D06068B0F551
:10927000803F17D0B0F5A02F286817D020F4803099
:109280002860286820F4802028606068E0B1FFF73B
:10929000ABFA804614E02868800322D56068002875
:1092A00078D01EE0286840F48030EDE740F480205C
:1092B0002860F7E7FFF798FAA0EB08006428A4D825
:1092C00028688003F6D50CE0FFF78EFA804605E0AB
:1092D000FFF78AFAA0EB0800642896D82868800374
:1092E000F6D4207880073BD5042E11D00C2E01D166
:1092F000022F0DD0E06801E0AAE1FFE00028286815
:109300001ED040F480702860FFF76EFA07460CE02C
:10931000286840050CD5E0680028C1D008E000BFEF
:10932000FFF762FAC01B022893D828684005F7D5DA
:109330006868217C20F0F85040EA016068600FE026
:1093400020F480702860FFF74FFA074605E000BF61
:10935000FFF74AFAC01B0228B1D828684005F7D4A5
:109360002078000729D560690028D5F8940012D02C
:1093700040F00100C5F89400FFF736FA074604E014
:10938000FFF732FAC01B022899D8D5F8940080075D
:10939000F6D512E02BE120F00100C5F89400FFF7AC
:1093A00023FA074605E000BFFFF71EFAC01B02289C
:1093B00085D8D5F894008007F6D42078400766D584
:1093C000A86D0027C00008D4A86D40F08050A865A3
:1093D000A86D012700F0805000904F480168C90532
:1093E00012D40168814641F480710160FFF7FCF9F5
:1093F000804605E0FFF7F8F9A0EB080002287DD8C9
:10940000D9F80000C005F5D5A068012816D00528B8
:10941000D5F8900017D020F00100C5F89000D5F8DD
:10942000900020F0040000BFC5F89000A06841F251
:109430008839C0B1FFF7D8F980460FE0D5F8900021
:1094400040F00100F0E740F00400C5F89000F5E7B7
:10945000FFF7CAF9A0EB080149454FD8D5F89000AD
:109460008007F5D50EE0FFF7BFF9804606E000BFA4
:10947000FFF7BAF9A0EB080149453FD8D5F89000AD
:109480008007F5D41FB1A86D20F08050A865207822
:10949000800628D5606A0028D5F8980012D040F0E0
:1094A0000100C5F89800FFF79FF9074605E000BFE7
:1094B000FFF79AF9C01B022820D8D5F8980080073A
:1094C000F6D510E020F00100C5F89800FFF78CF900
:1094D000074604E0FFF788F9C01B02280ED8D5F82C
:1094E00098008007F6D4A06AF0B3022816D00C2E9C
:1094F0007DD0286820F08070286000E0A7E0FFF7AA
:1095000073F90446A6E0000000100240E0FC0008E9
:10951000740000204C00002000700040E868E26AFF
:1095200000F00301914228D1216B00F07002090183
:109530001039914221D1626B00F4FE41B1EB022F50
:109540001BD194F8382000F07841B1EBC26F14D1F0
:10955000A18F00F4C00249084905A1F5001191420C
:109560000BD194F8401000E06AE04908490600F089
:10957000C060A1F1007181424BD00C2E73D02868DD
:10958000400170D4286820F080702860FFF72CF923
:10959000064604E0FFF728F9801B022857D8286800
:1095A0008001F7D4F4E90B016FF00F0202EB011117
:1095B0000843218A5204490802EB4151A26841EA5A
:1095C00002210843217D4FF07E42490802EB4161B0
:1095D0000843217B40EAC160E968244A11400843FE
:1095E000E860286840F080702860E86800E03AE0B1
:1095F00040F08070E860FFF7F7F8044605E000BF30
:10960000FFF7F2F8001B022821D828688001F7D55F
:1096100027E02868800124D4286840F08070286002
:10962000E86840F08070E860FFF7DEF8044604E088
:10963000FFF7DAF8001B022809D828688001F7D55F
:109640000FE000BFFFF7D0F8001B022802D903206B
:10965000BDE8F88328688001F4D4E868044908402C
:10966000E8600020F4E70120F2E700008C809D0113
:10967000FCFFEEFE7047704770470000F0B590F8B1
:109680003C20012A29D0012480F83C40022280F8A5
:109690003D2003685A689D68114EB34203D122F4FD
:1096A00070074A683A4322F070070A683A435A60E2
:1096B0000268B24205D0B2F1804F02D0094B9A4203
:1096C00004D1896825F080031943916080F83D40FA
:1096D000002180F83C100846F0BD0220F0BD0000DB
:1096E000002C01400040014010B5040003D094F864
:1096F0003D0010B107E0012010BD002084F83C00BF
:10970000204600F023F8022084F83D00211D206847
:1097100002F0F0FD012084F8480084F83E0084F84F
:109720003F0084F8400084F8410084F8420084F847
:10973000430084F8440084F8450084F8460084F827
:10974000470084F83D00002010BD00002DE9F04FD7
:1097500087B0064614216846FDF7F1F9454A31689D
:109760004548914263D1016E41F400610166016E8A
:1097700001F400610591C16C41F00101C164C06C4C
:109780004FF4807B00F00100CDF800B0059002207E
:109790000025CDE901050120CDE903505F4669466A
:1097A0004FF09040FEF730FF354C34484FF007083B
:1097B0002060C4E901854FF0800AE560C4E904A790
:1097C00007154FF02009A761C4E907952046FEF769
:1097D000FDFC08B1FDF7B1FE7462A662284C274873
:1097E000483414302060C4E9018504F10C01A761FC
:1097F00081E8200CC4E907952046FEF7E7FC08B194
:10980000FDF79BFEB462002205211A20A662FFF735
:109810007DF91A20FFF76DF9002205211B20FFF7C3
:1098200075F91B20FFF765F907B000F02FB8B1F10B
:10983000804F0BD0134A914210D1816D41F020012D
:109840008165806D00F020000590EDE7816D41F0AD
:1098500001018165806D00F00100F5E70A4A91423F
:10986000E2D1016E41F480310166006E00F4803077
:10987000EAE70000002C0140001002401C000240FA
:10988000DC170020001400400040014030BCBDE85F
:10989000C08F000090F83D10012901D001207047D1
:1098A000022180F83D100168CA6842F00102CA60D6
:1098B00000680B49884205D0B0F1804F02D00949B9
:1098C000884207D18168084A1140062906D0B1F5BF
:1098D000803F03D0016841F0010101600020704722
:1098E000002C0140004001400700010070B5044613
:1098F00090F83C000025012817D0012684F83C6030
:10990000022084F83D00226890682F4B184020F414
:109910007F4090600868502838D00DDC20284FD058
:1099200005DC90B3102811D14AE0022070BD302828
:1099300046D040280AD13BE060282FD070280DD0B7
:10994000B0F5805F03D0B0F5005F12D0012584F838
:109950003D60002084F83C00284670BDCB68D1E90A
:109960000121206802F086FD2068816841F07701BE
:1099700009E0CB68D1E90121206802F07BFD206875
:10998000816841F480418160E1E719E0CA68496873
:10999000206802F007FF5021206806E0CA68496885
:1099A000206802F039FF6021206802F06DFDCEE7EB
:1099B000CA684968206802F0F5FE40212068F4E793
:1099C000226801461046F0E788FFFEFF70477047A7
:1099D00070472DE9F041054690F83C0000260C4602
:1099E000012810D0012085F83C0072B1042A1CD057
:1099F000082A2CD00C2A50D00126002085F83C00E3
:109A00003046BDE8F0810220FBE7D4E90012E368AC
:109A1000286802F0D9FE2868816921F00C01816173
:109A200028688169A26811430FE0D4E90012E36855
:109A3000286802F003FF2868816921F44061816190
:109A400028688169A26841EA02218161D5E7286816
:109A5000D4E9002C277B016A21F480710162C1697D
:109A6000036A21F0030141EA0C0121F0F00C3907EF
:109A70004FF420674CEA116123F4206307EA0222C5
:109A80001A43C16102622868C16921F00C01C161F9
:109A90002868C169A268114328E02868D4E9002732
:109AA000E168036A23F480530362D0F81CC0036AA0
:109AB0002CF4407C4CEA07274FF6FF7C27F47047D4
:109AC0000CEA013139434FF4204723F4204307EADD
:109AD00002321A43C16102622868C16921F44061FF
:109AE000C1612868C169A26841EA0221C16184E7B5
:109AF00010B5040003D094F83D0010B107E0012038
:109B000010BD002084F83C00204600F022F802201E
:109B100084F83D00211D206802F0ECFB012084F850
:109B2000480084F83E0084F83F0084F8400084F840
:109B3000410084F8420084F8430084F8440084F82B
:109B4000450084F8460084F8470084F83D00002072
:109B500010BD70472DE9F0411F4690460D000446A8
:109B60004FF0000613D0042D16D0082D19D00C2D5F
:109B70001CD0102D1DD094F8430000BF94F847105E
:109B8000022819D0022917D0012818D0B4E094F87F
:109B90003E0094F84410F3E794F83F0094F8451021
:109BA000EEE794F8400094F84610E9E794F8410095
:109BB000E4E794F84200E1E70220BDE8F0810129E2
:109BC00078D1B8F1000F75D0002F73D002209DB36B
:109BD000042D37D0082D3AD00C2D3DD0102D3FD07C
:109BE00084F8430084F8470001222946206802F0E7
:109BF000B7FB45484549464A8DB3042D46D0082D4C
:109C000059D00C2D6AD0012642492068884205D0DF
:109C1000B0F1804F02D04049884207D181683F4A65
:109C20001140062906D0B1F5803F03D0016841F00C
:109C3000010101603046C0E7FFE784F83E0084F888
:109C40004400D1E784F83F0084F84500CCE784F86D
:109C5000400084F84600C7E784F84100C2E702E00C
:109C600084F84200BEE7636AD862606A3B460163DB
:109C7000606A4263216842463431606AFEF706FB3F
:109C8000C0B92068C16841F4007111E0A36AD862CC
:109C9000A06A3B460163A06A4263216842463831AC
:109CA000A06AFEF7F3FA28B92068C16841F4806120
:109CB000C160A9E720E0E36AD862E06A3B4601633D
:109CC000E06A4263216842463C31E06AFEF7DEFA10
:109CD00090B92068C16841F40061E9E7236BD8625C
:109CE000206B3B460163206B426321684246403152
:109CF000206BFEF7CBFA08B101205EE72068C1684F
:109D000041F48051D4E700007BC30008E9C3000898
:109D100021C40008002C0140004001400700010060
:109D200070B50446006801694FF00005C943890712
:109D300015D4C168C943890711D4E91E0161012006
:109D40002077206880698007204602D0FFF73FFE19
:109D500004E000F0CFF8204600F091F92577206864
:109D60000169C943490717D4C168C943490713D4D6
:109D70006FF004010161022020772068806910F4EF
:109D8000407F204602D0FFF722FE04E000F0B2F848
:109D9000204600F074F9257720680169C943090756
:109DA00016D4C168C943090712D46FF008010161D4
:109DB000042020772068C0698007204602D0FFF782
:109DC00006FE04E000F096F8204600F058F92577EA
:109DD00020680169C943C90617D4C168C943C906C7
:109DE00013D46FF010010161082020772068C0694A
:109DF00010F4407F204602D0FFF7E9FD04E000F0B8
:109E000079F8204600F03BF9257720680169C943BD
:109E1000C90708D1C168C943C90704D1891E0161B6
:109E2000204600F095F920680169C943090609D464
:109E3000C168C943090605D46FF08001016120465D
:109E4000FFF719FC20680169C943C90509D4C16835
:109E5000C943090605D46FF4807101612046FFF7FC
:109E600009FC20680169C943490609D4C168C9438E
:109E7000490605D46FF040010161204600F09DF9CC
:109E800020680169C94389060BD4C168C9438906A2
:109E900007D46FF0200101612046BDE87040FFF754
:109EA000EBBB70BD10B586B0044614216846FCF7C4
:109EB00046FE2068B0F1804F16D10C48C16C41F0CD
:109EC0000201C164C06C002100F0020005904FF453
:109ED000406000900220CDE9010103900120049030
:109EE00069460348FEF790FB06B010BD0010024023
:109EF00000040048704770B5044690F83C00002606
:109F00000D4601280BD0012084F83C000C2A4AD0D1
:109F100007DC82B1042A20D0082A06D131E00220D1
:109F200070BD102A53D0142A63D00126002084F873
:109F30003C00304670BD206802F0AEFA20688169AE
:109F400041F0080181612068816921F0040181618B
:109F5000206881692A69114311E0206802F0D8FA6B
:109F60002068816941F4006181612068816921F480
:109F700080618161206881692A6941EA02218161E9
:109F8000D4E7206802F000FB2068C16941F00801B5
:109F9000C1612068C16921F00401C1612068C16903
:109FA0002A69114311E0206802F028FB2068C1698A
:109FB00041F40061C1612068C16921F48061C1611F
:109FC0002068C1692A6941EA0221C161AEE72068BF
:109FD00002F044FB2068416D41F0080141652068B2
:109FE000416D21F0040141652068416D2A691143EA
:109FF00011E0206802F060FB2068416D41F40061CF
:10A0000041652068416D21F4806141652068416DA2
:10A010002A6941EA0221416588E710B5040003D0AE
:10A0200094F83D0010B107E0012010BD002084F835
:10A030003C00204600F022F8022084F83D00211D5B
:10A04000206802F057F9012084F8480084F83E00A7
:10A0500084F83F0084F8400084F8410084F842000E
:10A0600084F8430084F8440084F8450084F84600EE
:10A0700084F8470084F83D00002010BD7047704709
:10A0800010B50446022269B1042912D0082917D05C
:10A090000C291CD0102921D094F84300012824D089
:10A0A000012010BD94F83E000128F9D184F83E202B
:10A0B0001DE094F83F000128F2D184F83F2016E01B
:10A0C00094F840000128EBD184F840200FE094F888
:10A0D00041000128E4D184F8412008E094F84200CE
:10A0E0000128DDD184F8422001E084F843200122D8
:10A0F000206802F035F912492068124A884204D0DB
:10A10000904202D0104B984203D1436C43F4004379
:10A1100043642068884204D0B0F1804F01D090425F
:10A1200007D18168094A1140062906D0B1F5803F60
:10A1300003D0016841F001010160002010BD000062
:10A14000002C014000400140004401400700010094
:10A1500000680349884201D1FEF73CBC704700000B
:10A160000010004070B5044690F83C00012812D061
:10A17000012584F83C50022084F83D00204602F07E
:10A18000C9FA01004FF0000007D084F83D5084F870
:10A190003C00012070BD022070BD2168CA6822F019
:10A1A0004002CA602168CA6822F48042CA6084F80A
:10A1B0003D5084F83C00002070BD704770477047E8
:10A1C00070B50446806FE66F216889684FF010050E
:10A1D000090618D5212816D12068083050E8001F3C
:10A1E00021F0800140E80012002AF5D1E06E38B17C
:10A1F000FDF7F2FE20B1E06EFDF788FF202821D0A8
:10A20000204602F091FC20688068400618D5222E76
:10A2100016D12068083050E8001F21F0400140E8C6
:10A220000012002AF5D1206F38B1FDF7D5FE20B11C
:10A23000206FFDF76BFF202804D0204602F04FFC72
:10A24000002070BDC4F88050032070BD70B50400BC
:10A2500019D02420A0672068016821F00101016065
:10A2600020680025056020684560206885602046DC
:10A2700000F08AF9C4F88050A567E56744F8605F8C
:10A280000020257570BD012070BD70472DE9F0419B
:10A2900002680446D0691168936840F60F052842A9
:10A2A0004FF0000505D186067ED58E067CD5616E01
:10A2B0001BE1994F03F001060F40374374D0C707E5
:10A2C00009D0CF0507D501271762D4F8802042F0C6
:10A2D0000102C4F8802082070AD5DA0708D027686F
:10A2E00002223A62D4F8802042F00402C4F88020AE
:10A2F00042070AD5DA0708D0236804221A62D4F884
:10A30000802042F00202C4F8802002070CD501F040
:10A310002002324308D0236808221A62D4F8802031
:10A3200042F00802C4F8802002050BD54A0109D585
:10A3300023684FF400621A62D4F8802042F02002B1
:10A34000C4F88020D4F88020002A35D0800605D5B6
:10A35000880603D5616E09B120468847D4F880008D
:10A3600021688968490602D410F0280F26D02046BB
:10A3700002F0B5FB2068806840061AD520680830D6
:10A3800050E8001F21F0400140E80012002AF5D1FA
:10A39000206F70B161498163206FFDF742FE002894
:10A3A0000AD0206F816B01E00EE02046BDE8F0414D
:10A3B00008472046FFF769FFBDE8F0812046FFF718
:10A3C00064FFC4F88050F7E7276E2026012F7BD169
:10A3D000C70679D5CF0677D510201062206880682F
:10A3E000400641D5216F086840680004000CE3D0A6
:10A3F000B4F858208242DFD9A4F85A0008680068EF
:10A4000080062AD4206850E8001F21F4807140E8BB
:10A410000012002AF6D12068083050E8001F21F011
:10A42000010140E80012002AF5D12068083050E808
:10A43000001F21F0400140E80012002AF5D1E66734
:10A440002566216851E8000F20F0100041E8000265
:10A45000002AF6D1206FFDF7BFFDB4F85800B4F81C
:10A460005A10401A81B22AE0B4F85800B4F85A10D1
:10A47000401A81B2B4F85A0000289DD000299BD020
:10A48000226852E8000F20F4907042E80003002B8D
:10A49000F6D12068083050E8002F22F0010240E891
:10A4A0000023002BF5D1E66725666566226852E831
:10A4B000000F20F0100042E80003002BF6D12046E8
:10A4C000FFF77CFE78E7FFE7C70209D55B0207D5F7
:10A4D0004FF4801010622046BDE8F041FFF76FBED8
:10A4E000020606D50A0604D5A16E00297FF45DAFE9
:10A4F00062E74006E6D54806E4D52046026852E801
:10A50000001F21F0400142E80013002BF6D18667BE
:10A51000856600F021FA4FE72001000497C9000882
:10A5200010B5040002D0A06F10B107E0012010BDEB
:10A53000002084F87400204600F058F82420A0671A
:10A540002068016821F001010160204602F0F8FA5C
:10A550000128ECD0606A10B1204602F08AF9206828
:10A56000416821F4904141602068816821F02A010E
:10A5700081602068016841F0010101602046BDE86A
:10A58000104002F0DAB9000010B50446144B01681F
:10A5900014484FF09042994213D1016E21F480414A
:10A5A00001664FF4C0611046FDF78CFF206FFDF788
:10A5B0005FFDE06EFDF75CFDBDE810402520FEF775
:10A5C00087BA094B99420AD1816D21F40031816526
:10A5D000BDE8104048F204011046FDF773BF10BDFE
:10A5E0000038014000100240004400402DE9F047CF
:10A5F0009EB00746142117A8FCF7A1FA5C21684613
:10A60000FCF79DFA4D4938684D4D002402264FF065
:10A6100003084FF007094FF0904A88425AD10120B1
:10A62000009008946846FEF7DFFA08B1FCF785FF52
:10A63000286E40F480402866286E00F480401C900C
:10A64000E86C40F00100E864E86C19AA00F0010031
:10A650001C904FF4C060CDE9170682E8100317A9DB
:10A660005046FDF7D1FF384D36484FF0800828603E
:10A67000C5E90164C5E903486C61AC61EC61284639
:10A680002C62FDF7A3FD08B1FCF757FF3D67AF62F1
:10A690002D4D2C4848351438E5E802061020A5E871
:10A6A0001101294845F814494830AC61EC612C622D
:10A6B000FDF78CFD08B1FCF740FFFD660022052187
:10A6C0002520AF62FEF722FA2520FEF712FA1EB00F
:10A6D000BDE8F0871D498842F9D168460096099483
:10A6E000FEF782FA08B1FCF728FFA86D40F40030AD
:10A6F000A865A86D00F400301C90E86C40F00100E3
:10A70000E864E86C19AA00F001001C900420CDE96F
:10A710001706454682E8300217A957465046FDF70E
:10A7200073FFCDE919454FF400401B95CDE917069D
:10A7300017A93846FDF768FFC9E700000038014057
:10A7400000100240580002407419002000440040EC
:10A7500030B4C36F202B20D1E1B1DAB190F874305E
:10A76000012B1AD0012380F87430002303660C4CAF
:10A770000368A3420BD05B681B0208D5046854E849
:10A78000003F43F0806344E80035002DF6D130BC33
:10A7900002F0D6BA012030BC70470220FBE700006F
:10A7A0000080004010B500681149ADF5187D884261
:10A7B0001BD1002096904FF496720E496846FCF724
:10A7C000A5F90D4C002396AA6946206804F08CFE7A
:10A7D00001280AD096AA4BA9206804F081FF002323
:10A7E00096AA6946206804F07FFE0DF5187D10BD1D
:10A7F00000380140041A002040000020704700008B
:10A800002DE9F8430446806F1F4616460D46202862
:10A810004FD1CDB1C6B194F87400012849D00120C0
:10A8200084F874004FF00008C4F880802120A067ED
:10A83000FDF7DAFFA4F850608146A4F85260A068E2
:10A84000B0F5805F03D004E00120BDE8F883206903
:10A8500028B12E465FF0000584F8748010E00026D1
:10A86000FAE78021204602F0BDFAB8B9C6B116F861
:10A87000010B21680885B4F85200401EA4F852006C
:10A88000B4F852004B464FF0000200970028E8D180
:10A890004FF04001204602F0A5FA30B10320D4E782
:10A8A00035F8020BC0F30800E3E72020A067002082
:10A8B000CBE70220C9E7000070B50446806F20286E
:10A8C00041D169B362B394F8740001283BD00120F0
:10A8D00084F87400E164A4F85020A4F85220002504
:10A8E000C4F880502120A067E06ED8B11749C1623A
:10A8F000E16E174813460863E16E16484863E06E40
:10A9000085632668E16C06F12802E06EFDF7BEFC67
:10A9100040B11020C4F8800004F8745F202060600B
:10A92000012070BD21684020086284F874502068BE
:10A93000083050E8001F41F0800140E80012002A72
:10A94000F5D1002070BD022070BD000093CA000840
:10A95000D5CA0008ABC9000800680449884204D180
:10A96000002220210248FDF73ABF7047003801401D
:10A97000000400487047FEE700241A4F1A4E25468F
:10A98000307850B101280AD002280AD003280AD012
:10A9900000203978032908D008E00220F9E70320D5
:10A9A000F7E70420F5E70520F3E706207178012991
:10A9B00000D10720A04202D0044602F0BFFA0B48A3
:10A9C00000F01AF80A4800F017F8642D04D9094974
:10A9D00000250888401C08800A206D1C03F006FA38
:10A9E000CEE700002401002000000020C400002069
:10A9F000B00000208001002010B50446807A0028B5
:10AA000032D0E288002A2FD020890A3081B22181F9
:10AA1000A37C002053B1E289914225D32081207389
:10AA2000A074E074A188002220680BE091421BD33F
:10AA30002081E07C50B10020E0740028A1882068CB
:10AA400006D00122BDE81040FDF7C9BE0120F3E7A2
:10AA50000022FDF7C4FE207B401CC0B22073E17AC7
:10AA6000884201D30120A07410BD00EB8100006E6C
:10AA700000F0F84070478068C0F3C00070478068FD
:10AA8000C0F380007047C06810F4406F01D0002010
:10AA9000704701207047042303EAD15310B51844CE
:10AAA0004369C1F3045107248C40A3438A401343F4
:10AAB000436110BD00EB8100016E21F000411143A4
:10AAC000016670477CB50C46054608221031684681
:10AAD000FCF71AFD208AC0F3C500382802D2C0F165
:10AAE000380201E0C0F178020749204600F02EFC50
:10AAF00008226946204600F029FC102221462846FB
:10AB0000FCF702FD7CBD00003CFD00080021416116
:10AB1000016105490160054941600349C9438160FC
:10AB20000249C943C16070470123456789ABCDEF36
:10AB30002DE9F043054691B055F8049B402295E875
:10AB4000D00068462D1FFBF7E1FF04EA060027EA64
:10AB500004010843FE49009A014402EB090008443D
:10AB600004EB706000EA040126EA00021143F94A8E
:10AB70001144019A3A44114400EB315101EA0002B8
:10AB800024EA01031A43F44B1A44029B33441A4447
:10AB900001EBF23202EA010320EA020C43EA0C0361
:10ABA000DFF8B8C36344DDF80CC0A444634402EB8F
:10ABB000B32303EA020C21EA03084CEA080CDFF88D
:10ABC000A083C444DDF810804044604403EB70600F
:10ABD00000EA030C22EA00084CEA080CDFF8848340
:10ABE000C444DDF814804144614400EB315101EA72
:10ABF000000C23EA01084CEA080CDFF86C83C4441B
:10AC0000DDF818804244624401EBF23202EA010CA2
:10AC100020EA02084CEA080CDFF85083C444DDF84F
:10AC20001C804344634402EBB32303EA020C21EA91
:10AC300003084CEA080CDFF83883C444DDF82080B0
:10AC40004044604403EB706000EA030C22EA000811
:10AC50004CEA080CDFF81C83C444DDF8248041442E
:10AC6000614400EB315101EA000C23EA01084CEA8F
:10AC7000080CDDF82880ACF5244C4244ACF14F0CB4
:10AC8000624401EBF23202EA010C20EA02084CEACB
:10AC9000080CDFF8E482C444DDF82C8043446344AC
:10ACA00002EBB32303EA020C21EA03084CEA080C86
:10ACB000DFF8C882C444DDF830804044604403EBD0
:10ACC000706000EA030C22EA00084CEA080CDFF886
:10ACD000B082C444DDF834804144614400EB31511A
:10ACE00001EA000C23EA01084CEA080CDFF8948220
:10ACF000C444DDF838804244624401EBF23202EA97
:10AD0000010C20EA02084CEA080CDFF87C82C444FB
:10AD1000DDF83C804344634402EBB32303EA010CB7
:10AD200022EA01084CEA080CDFF86082C444DDF82E
:10AD300004804044604403EBF06000EA020C23EA24
:10AD400002084CEA080CDFF84882C444DDF8188099
:10AD50004144614400EBF15101EA030C20EA03088D
:10AD60004CEA080CDFF82C82C444DDF82C80424405
:10AD7000624401EBB24202EA000C21EA00084CEA0C
:10AD8000080CDFF81482C444DDF8008043446344B7
:10AD900002EB333303EA010C22EA01084CEA080C07
:10ADA000DFF8F881C444DDF814804044604403EBCC
:10ADB000F06000EA020C23EA02084CEA080CDFF813
:10ADC000E081C444DDF828804144614400EBF15146
:10ADD00001EA030C20EA03084CEA080CDFF8C481FE
:10ADE000C444DDF83C804244624401EBB24202EAD2
:10ADF000000C21EA00084CEA080CDFF8AC81C444DE
:10AE0000DDF810804344634402EB333303EA010C62
:10AE100022EA01084CEA080CDFF89081C444DDF80E
:10AE200024804044604403EBF06000EA020C23EA13
:10AE300002084CEA080CDFF87881C444DDF8388059
:10AE40004144614400EBF15101EA030C20EA03089C
:10AE50004CEA080CDFF85C81C444DDF80C80424405
:10AE6000624401EBB24202EA000C21EA00084CEA1B
:10AE7000080CDFF84481C444DDF820804344634477
:10AE800002EB333303EA010C22EA01084CEA080C16
:10AE9000DFF82881C444DDF834804044604403EB8B
:10AEA000F06000EA020C23EA02084CEA080CDFF822
:10AEB0001081C444DDF808804144614400EBF15145
:10AEC00001EA030C20EA03084CEA080CDFF8F480DE
:10AED000C444DDF81C804244624401EBB24C0CEAED
:10AEE000000221EA000842EA0802DFF8DC8042445E
:10AEF000DDF8308043441A440CEB3233059ADFF816
:10AF0000CC80104483EA0C024A4042441044089A20
:10AF100003EB3070114480EA030282EA0C02DFF88E
:10AF2000B080424411440B9A00EB7151624481EAB3
:10AF3000000CDFF8A0808CEA030CC4446244DDF806
:10AF400038C001EB3242634482EA010C44E0000065
:10AF500078A46AD756B7C7E8DB702024EECEBDC10F
:10AF6000AF0F7CF52AC68747134630A8019546FDEA
:10AF7000D8988069AFF7448BBED75C892211906B5B
:10AF8000937198FD8E4379A62108B44962251EF677
:10AF900040B340C0515A5E26AAC7B6E95D102FD60D
:10AFA0005314440281E6A1D8C8FBD3E7E6CDE121E2
:10AFB000D60737C3870DD5F4ED145A4505E9E3A943
:10AFC000F8A3EFFCD9026F678A4C2A8D4239FAFF49
:10AFD00081F6718722619D6DDFF8FC828CEA000C9E
:10AFE000C4446344DDF804C002EB7323604483EA85
:10AFF000020CDFF8E8828CEA010CC4446044DDF8FE
:10B0000010C003EB3070614480EA030CDFF8D0829B
:10B010008CEA020CC4446144DDF81CC000EB7151A1
:10B02000624481EA000CDFF8BC828CEA030CC44461
:10B030006244DDF828C001EB3242634482EA010C2D
:10B04000DFF8A4828CEA000CC4446344DDF834C009
:10B0500002EB7323604483EA020CDFF890828CEAEF
:10B06000010CC4446044DDF800C003EB307061445F
:10B0700080EA030CDFF878828CEA020CC444614455
:10B08000DDF80CC000EB7151624481EA000CDFF87E
:10B0900064828CEA030CC4446244DDF818C001EBFE
:10B0A0003242634482EA010CDFF84C828CEA000CE5
:10B0B000C4446344DDF824C002EB7323604483EA94
:10B0C000020CDFF838828CEA010CC4446044DDF8DD
:10B0D00030C003EB3070614480EA030CDFF820825B
:10B0E0008CEA020CC4446144DDF83CC000EB7151B1
:10B0F000624481EA000CDFF80C828CEA030CC44441
:10B100006244DDF808C001EB3242634482EA010C7C
:10B11000DFF8F4818CEA000CC4446344DDF800C01D
:10B1200002EB7323604463EA010CDFF8E0818CEAF0
:10B13000020CC4446044DDF81CC003EBB060614401
:10B1400060EA020CDFF8C8818CEA030CC444614455
:10B15000DDF838C000EBB151624461EA030CDFF85E
:10B16000B4818CEA000CC4446244DDF814C001EBE5
:10B170007242634462EA000CDFF89C818CEA010CA5
:10B18000C4446344DDF830C002EBF323604463EA57
:10B19000010CDFF888818CEA020CC4446044DDF8BD
:10B1A0000CC003EBB060614460EA020CDFF8708110
:10B1B0008CEA030CC4446144DDF828C000EBB151B3
:10B1C000624461EA030CDFF85C818CEA000CC44441
:10B1D0006244DDF804C001EB7242634462EA000C91
:10B1E000DFF844818CEA010CC4446344DDF820C0DC
:10B1F00002EBF323604463EA010CDFF830818CEA50
:10B20000020CC4446044DDF83CC003EBB060614410
:10B2100060EA020CDFF818818CEA030CC444614434
:10B22000DDF818C000EBB151624461EA030CDFF8AD
:10B2300004818CEA000CC4446244DDF834C001EBA4
:10B240007242634462EA000CDFF8EC808CEA010C85
:10B25000C4446344DDF810C002EBF323604463EAA6
:10B26000010CDFF8D8808CEA020CC4446044DDF89D
:10B270002CC003EBB060614460EA020CDFF8C080D0
:10B280008CEA030CC4446144DDF808C000EBB15102
:10B29000624461EA030CDFF8AC808CEA000CC44421
:10B2A0006244DDF824C001EB7242634462EA000CA0
:10B2B0008CEA010CDFF890804844C444634402EBFC
:10B2C000F3232860E0186860B018A8607818E86078
:10B2D00011B0BDE8F08300000C38E5FD44EABEA4DF
:10B2E000A9CFDE4B604BBBF670BCBFBEC67E9B28B1
:10B2F000FA27A1EA8530EFD4051D880439D0D4D9C6
:10B30000E599DBE6F87CA21F6556ACC4442229F41B
:10B3100097FF2A43A72394AB39A093FCC3595B65DD
:10B3200092CC0C8F7DF4EFFFD15D84854F7EA86FAA
:10B33000E0E62CFE144301A3A111084E827E53F7D0
:10B3400035F23ABDBBD2D72A91D386EB2DE9F04135
:10B350000F46016905461646C1F3C50001EBC6015B
:10B360002961B1EBC60F696901D2491C696101EB22
:10B370005671C0F140046961A64216D328442246A2
:10B3800039461830FBF7C2FB05F118012846FFF7D4
:10B39000CFFB04E039192846FFF7CAFB403404F11B
:10B3A0003F00B042F6D3002000E00024321B3919E0
:10B3B0002844BDE8F0411830FBF7A8BB10B586B0B3
:10B3C00018216846FBF7BBFB3148304900F10C03FC
:10B3D00001600021416001220424816083E816009D
:10B3E000017642760523C36180F820108162C16234
:10B3F00080F830201203426380F83810FCF746FCD6
:10B4000008B1FCF79AF82348009006200190072025
:10B4100002907F2003900320CDE9040469461C4874
:10B42000FCF738FA08B1FCF788F81B4800900C20AC
:10B43000019069461648FCF72DFA08B1FCF77DF833
:10B44000164800901220019069461148FCF722FA34
:10B4500008B1FCF772F81248009018200190694674
:10B460000B48FCF717FA08B1FCF767F80D48009095
:10B470004FF48070019069460548FCF70BFA0028EC
:10B4800001D0FCF75AF806B010BD000000000450CF
:10B49000AC1500200002B0250004002A0008302E60
:10B4A0000010603200002143194808B5816C41F05A
:10B4B00001018164806C002200F0010000900521F0
:10B4C0000B20FDF723FB0B20FDF713FB00220521CA
:10B4D0000C20FDF71BFB0C20FDF70BFB00220521C8
:10B4E0000D20FDF713FB0D20FDF703FB00220521C6
:10B4F0000E20FDF70BFB0E20FDF7FBFA00220521C5
:10B500000F20FDF703FBBDE808400F20FDF7F1BA5F
:10B510000010024010B51CA001F0E6FD1E4C0220F8
:10B52000607002F003FC1D48008900F037FE00F057
:10B53000FFFD1B4A4FF49671102002F093FC184A4D
:10B540002064B43A0021174802F0B8FC144AE062C3
:10B55000903A0021144802F0B1FC114A20636C3A81
:10B560000021124802F0AAFC0D4A6063483A00210B
:10B570000F4802F0A3FC0A4AA063243A00210D48B8
:10B5800002F09CFCE06310BD415049325F454C45E0
:10B5900020303631320D0A00000000203802002031
:10B5A000C8FC000879A9000839BF0008FB7400082E
:10B5B0004573000865B900082DE9F04186B01421F3
:10B5C0006846FBF7BCFA2348C16C41F00101C16435
:10B5D000C16C01F001010591C16C41F00201C1642F
:10B5E000C06C1D4F00F002000590012241F20401E1
:10B5F0003846FDF7F4F84FF4C0564FF0904800225B
:10B6000031464046FDF7EBF80022E0213846FDF7D1
:10B61000E6F8E420009001250024CDE901546946B4
:10B6200038460394FCF7F0FF2803CDE9000503201A
:10B63000CDE9024069463846FCF7E6FF0096CDE9C1
:10B640000154694640460394FCF7DEFF06B0BDE8AE
:10B65000F08100000010024000040048134810B5BB
:10B66000114901601249416000210122C0E9021222
:10B67000016141618161C1610162FDF70FF908B1AA
:10B68000FBF75BFF00210948FDF7B4F808B1FBF7B1
:10B6900054FF00210548FDF7D8F8002803D0BDE885
:10B6A0001040FBF74ABF10BD00580040581600205C
:10B6B000694EA53010B588B0002418480094019454
:10B6C00002940394049405941349069401604F2155
:10B6D000C0E901144FF6FF71C0E9031444618461AD
:10B6E000FEF702F808B1FBF728FF4FF480500090F6
:10B6F00069460A48FEF7FAF808B1FBF71EFF049402
:10B7000004A906480694FDF7B9FF002801D0FBF70D
:10B7100014FF08B010BD0000004001409017002049
:10B7200010B590B000240C940D940E94142104A82C
:10B730000F94FBF704FA2E480A940B940994009492
:10B74000019402942949039401604F21C0E9011436
:10B750004FF6FF71C0E903148021C0E90541FDF7F0
:10B76000C3FF08B1FBF7E9FE4FF480500C900CA921
:10B770001F48FEF7BBF808B1FBF7DFFE1C48FEF7D9
:10B78000B7F908B1FBF7D9FE042004905020CDE9A9
:10B79000050404A916480894FEF7E4FC08B1FBF779
:10B7A000CCFE09940A9409A911480B94FDF766FF91
:10B7B00008B1FBF7C2FE0120CDE90040029400224F
:10B7C00069460B480394FEF704F908B1FBF7B5FE90
:10B7D000022000900190042269460548FEF7F9F81E
:10B7E000002801D0FBF7A9FE10B010BD002C0140CD
:10B7F000AC16002010B58EB000240794089409946C
:10B800000A940B940C941C2168460D94FBF797F94D
:10B8100022484FF0804101602721C0E9011440F225
:10B82000E731C0E903148461FDF75EFF08B1FBF75F
:10B8300084FE4FF48050079007A91848FEF756F889
:10B8400008B1FBF77AFE1548FEF7E7FB08B1FBF7F6
:10B8500074FE0B940BA911480D94FDF70FFF08B16E
:10B86000FBF76BFE602000904FF4FA70CDE9010405
:10B870000822694609480494FEF73DFB08B1FBF72E
:10B880005CFE0C2269460548FEF735FB08B1FBF764
:10B8900054FE0248FEF706FB0EB010BDF81600205D
:10B8A0003EB500240F48009401940D4902940160B4
:10B8B0004F21C0E901144FF6FF718461C160FDF7AB
:10B8C00013FF08B1FBF739FE00946946054802945E
:10B8D000FDF7D4FE002801D0FBF72FFE3EBD00008F
:10B8E00000140040441700200D4810B50B490160BA
:10B8F0004FF416514160002181600C22C160C0E903
:10B9000004128161C16101624162FEF709FE0028F3
:10B9100003D0BDE81040FBF710BE10BD0038014059
:10B920006C1800200D4810B50B4901604FF47A31B6
:10B930004160002181600C22C160C0E90412816174
:10B94000C16101624162FEF7EBFD002803D0BDE852
:10B950001040FBF7F2BD10BD00440040F01800207D
:10B96000FEE7000008213C48FEF78AFB0C213A481C
:10B97000FEF786FB002600F0D1F8DFF8E090DFF854
:10B98000E0B0384FDFF8D080002400BF99F8000005
:10B99000A8B33549F868884210DD40F2DC50864291
:10B9A00002D20A36B6B20AE003218BF80010D8F8AA
:10B9B0000010CC63D8F80000046400E00026DFF833
:10B9C000ACA0D7ED040A50469AED020A00F067F8E1
:10B9D000BDEEC00A40F2BA2110EE100A05B205F21F
:10B9E0005D1088420DD89AED020AB5EEC00AF1EE5C
:10B9F00010FA06D0002D03DD4FF4FA7501E018E0CF
:10BA00001B4D9BF80000DA46012802D1A8B200F0D5
:10BA100031F89AF80000022802D1A8B200F034F8F8
:10BA20009AF8000028B9D8F80010CC63D8F80000C4
:10BA30000464387840B1D8F800100C64022806D0AD
:10BA4000032804D0012802D0D8F80000C4630A20DB
:10BA500002F0CCF99AE70000F81600201801002047
:10BA60002401002000000020295C0F3D881B0020DD
:10BA70000CFEFFFF03490A68D063096800200864D0
:10BA800070470000F8160020034900220B68DA63B3
:10BA90000968086470470000F8160020FEE730EEE1
:10BAA000600AB0EE002A80ED030AD0ED040AD0ED62
:10BAB000071A30EE601A21EE211AD0ED081A01EEB5
:10BAC000801AD0ED061A70EE211A40EEC21A90EDDF
:10BAD000092A02EE211AD0ED0A1A31EE211A80ED60
:10BAE0000A1AC0ED060A80ED040A90ED0B0AB4EEC6
:10BAF000C01AF1EE10FA01DD80ED0A0AD0ED0A0A53
:10BB0000B1EE400AF4EEC00AF1EE10FA02D3B0EE44
:10BB1000600A704780ED0A0A7047000015489FEDE3
:10BB2000140ADFED150A80ED000A80ED010AC0ED70
:10BB3000020A80ED030A80ED040A80ED050A9FEDFC
:10BB40000F0A80ED070A9FED0E0A80ED080A9FEDAF
:10BB50000D0A80ED090A9FED0C0A80ED0B0A9FED9E
:10BB60000B0A80ED0C0AB1EE040A80ED0D0A704755
:10BB700000000000881B0020000048436666A63FC6
:10BB80003333333FCDCC4C3E00007A4400007AC4BE
:10BB900070B52DED048BFCF727FE05465448406A2E
:10BBA000006840680A21C0F10A00B0FBF1F201FB15
:10BBB00012005049504A51F8201052F82000002835
:10BBC0006FD000EE101AF8EE400A00EE100AB8EE40
:10BBD000401A80EE810ADFED490A20EE200A9FED2F
:10BBE000481A484C20EE018A94ED060A9FED461A49
:10BBF00000EE018A84ED028A206A281A01EE100AFA
:10BC0000B8EE411ADFED411A4149C1EE218A18EE22
:10BC1000900A884269DD38EE400A3E49C4ED058A43
:10BC200010EE100A884202DD30EE600A06E010EEE7
:10BC3000100A3949884201D930EE200AB2EE049A3E
:10BC400020EE090A01F070FAC0EE090A3349B0EE9D
:10BC5000E00A10EE100A884202DAC0EEA82A01E0DB
:10BC6000D4ED092A94ED090A2D4972EEC00AF0EECE
:10BC7000E00A10EE900A884201DDF0EE402A2948E1
:10BC80000078012802D002280CD015E0F5EEC02A79
:10BC9000F1EE10FA02D2D4ED0A2A0DE0C4ED0A2A20
:10BCA0000AE022E0F5EEC02AF1EE10FA02DDD4ED52
:10BCB0000B2A01E0C4ED0B2A18EE100A1A490844B9
:10BCC0001A49884206D318EE100A1949084419493E
:10BCD000884201D2F0EE402AB0EE620A01F092F9F9
:10BCE000C4ED092A256284ED068ABDEC048B70BD83
:10BCF000AC160020740200204C0200200000B44367
:10BD0000CDCC4C3E78000020CDCC4C3F00007A4496
:10BD10006F12833A00003443000034C300007042C5
:10BD20000000C84324010020FFFF8FBEFFFFEB008F
:10BD3000FFFF50BC32F3040000B5CBB04FF4967156
:10BD40006846FAF7FCFE114800226946006803F0D5
:10BD50002BFC012807D1684601F074FF00286846D3
:10BD600003D002F01DF94BB000BD01F08FFF002899
:10BD7000684602D002F05AF9F5E701F0ABFF00285F
:10BD8000F1D0684602F06CFAEDE7000040000020B8
:10BD90002DE9F041444C05468846E06800268107BD
:10BDA00028680DD0E16801F00301814216D1A8B1E5
:10BDB000E0686968C0F30210401C88420ED120E0A0
:10BDC000012804D0022805D0032807D108E0216803
:10BDD000890701E021684905002907DB01265FE0AA
:10BDE0002168890302D421684903F5E7E1686A689C
:10BDF0006FF00F0321F0730103EB021211430143B3
:10BE0000E160206820F080602060FCF7EDFC0746D0
:10BE100005E000BFFCF7E8FCC01B022837D820680B
:10BE20000001F7D4B8F1000F18D0B8F1010F1DD000
:10BE3000287D4FF07E41400801EB4060A96840EA50
:10BE400001202169194A114008432061206840F00F
:10BE500080602060FCF7C8FC07461AE0A868297BD0
:10BE6000000240EAC1602169114AECE7288A1149C1
:10BE7000400801EB4050A96840EA012021690E4AC0
:10BE8000E1E700BFFCF7B0FCC01B022801D9032684
:10BE900006E020680001F5D52069A9690843206102
:10BEA0003046BDE8F081000000100240FF80FFF93D
:10BEB000FF80FF070000E0FFFF809FFFF8B51C4DEB
:10BEC00006460024A86DC00002D5FCF785FE0DE0F3
:10BED000A86D40F08050A865A86D00F080500090DB
:10BEE000FCF77AFEA96D21F08051A965B0F5007FBD
:10BEF00004D0802E07D94FF003040AE0802E08D921
:10BF0000A02E01D804E001D1022402E0702E00D15D
:10BF100001240848016821F00701214301600068FD
:10BF200000F00700A04201D00120F8BD0020F8BDBC
:10BF300000100240002002402DED048B0A23002156
:10BF40006A4A6B48FDF706FE684A0A232832042134
:10BF50006748FDF7FFFD6748FBF79CF97F216548BF
:10BF6000FBF750FC6149052220396248FBF7DAFFF4
:10BF70005E4D203D9FED608ADFED608ADFF880A195
:10BF8000DFF88091604FDFF88481614C614EB0EE44
:10BF9000009A4FF0010B00BF01F0D4FF01F0E6FF63
:10BFA0002B88A38000EE103A6A88E280B8EE400A3F
:10BFB000A9882181E88820EE080A6081B5F808C0C8
:10BFC000A4F802C020EE280A84ED050A00EE102A2B
:10BFD000B8EE400A20EE080A20EE280A84ED060A90
:10BFE00000EE101AB8EE400A20EE080A20EE280AE9
:10BFF00084ED070A00EE100AB8EE400A20EE080AA7
:10C0000020EE280A84ED080A00EE10CAB8EE400AB5
:10C0100020EE080A20EE280A10EE100A84ED090A24
:10C02000504503DD9FED3C0A84ED090A20EE090A24
:10C0300084ED0A0A84ED030A01F0A2FF01F08CFFEF
:10C040006069414600EB09038B420CD2A369BB42F5
:10C0500009DDDFF8C8C0236A634504DDB3F17F5F03
:10C0600001DA00200EE000EB09028A420DD2A2693B
:10C07000BA420ADD226AB2F17F5F06DDB2F1804F7B
:10C0800003DA5846207030802CE04FF07E539842FF
:10C090000FDAA2699A420CDD214B9A4209DA194B58
:10C0A000226ADB439A4204DDB2F1804F01DA0220BA
:10C0B00015E01C4A1044404510D21B49A069884233
:10C0C0000CDD1A49884209DA0E49206AC9438842C0
:10C0D00004DDB0F1804F01DA032000E0042020707D
:10C0E000A6F800B0052001F081FE55E74C020020C3
:10C0F000AC160020AC1500200000803933335340CB
:10C1000033335340323333C00000204032333300E6
:10C11000000000208201002000000000CDCC8C3FF8
:10C120003333B33F656666C06666663F6666A63FA4
:10C1300070B50E48FEF744F80C4C2068016821F0F9
:10C14000100101600A4900204FF4967508802946C5
:10C150000848FAF7F4FC2A4606492046FEF7F8FAA2
:10C160002068016841F01001016070BD6C1800206A
:10C1700044000020041A002010B5064C012120467E
:10C18000FBF784FA2046BDE8104007220249FBF77E
:10C190001BBB000000680308E01C002010B54FF432
:10C1A000165109281AD2DFE800F0190519080B0EFC
:10C1B000111417004FF4965110E04FF496410DE022
:10C1C0004FF416410AE04FF4614107E04FF4E131CA
:10C1D00004E04FF4613101E04FF47A310F480E4A28
:10C1E000C0E90021002181600C22C160C0E9041275
:10C1F0008161C16101624162FEF728F808B1FBF775
:10C200009CF90648FEF78CF9002803D0BDE81040E1
:10C21000FBF793B910BD0000003801406C180020F6
:10C2200010B54FF0E020006903F03EFB012803D079
:10C23000BDE8104002F0FABF10BD00B597B0442130
:10C240006846FAF77CFC142111A8FAF778FC4FF441
:10C250000070FCF78DFC08B172B6FEE70220C10148
:10C2600003911021009004910A900121CDE90B0166
:10C270000A210D910721CDE90E1010906846FCF7B8
:10C2800049FF08B172B6FEE70F201190032012900B
:10C290000020139014901590042111A8FCF702FEC1
:10C2A000002801D072B6FEE717B000BD0248016851
:10C2B00041F470010160704788ED00E010B5064858
:10C2C000FDF72EFD002201211B20FCF71FFCBDE81D
:10C2D00010401B20FCF70DBCAC1600200148FDF7F8
:10C2E0001FBD0000AC1600200148FDF719BD00007D
:10C2F000301B002070B50268164B4FF08046984204
:10C3000001D0B04203D122F070044A682243124C9B
:10C31000124D984205D0B04203D0A04201D0A842AD
:10C3200003D122F44076CA6832434E6922F080027B
:10C33000324302608A68C2620A688262984203D00D
:10C34000A04201D0A84201D10969016301214161E4
:10C3500070BD0000002C014000400140004401403D
:10C3600010B501F01F030121046A99408C43046257
:10C37000016A9A401143016210BD10B5846A01211F
:10C38000626A824207D12177C06938BB84F83E10C7
:10C3900084F8441022E0A26A824208D10222227765
:10C3A000C069D8B984F83F1084F8451016E0E26AF5
:10C3B000824208D104222277C06978B984F84010FB
:10C3C00084F846100AE0226B824207D108222277C5
:10C3D000C06918B984F8411084F847102046FDF769
:10C3E000F6FA0020207710BD10B5846A616A814298
:10C3F00001D101200DE0A16A814201D1022008E0B3
:10C40000E16A814201D1042003E0216B814201D124
:10C41000082020772046FDF7DBFA0020207710BDAA
:10C4200010B5846A0121626A824203D1217784F8BF
:10C430003E1019E0A26A824204D10220207784F8DB
:10C440003F1011E0E26A824204D10420207784F890
:10C45000401009E0226B824204D10820207784F842
:10C46000411001E084F83D102046FDF7AFFA0020AE
:10C47000207710BD10B5846842EA032224F47F447B
:10C480000A432243826010BD826822F070020A4390
:10C4900042F0070181607047F0B5026A22F00102A4
:10C4A0000262056A43688269154C25F00205224044
:10C4B0000C6822F0030214438A68134E2A43114D7C
:10C4C000124FA84203D0B04201D0B84206D122F0A8
:10C4D000080CCA6842EA0C0222F00402A84203D007
:10C4E000B04201D0B84205D14D6923F440731D43D9
:10C4F0008B692B4343608461496841630262F0BDEC
:10C500008FFFFEFF002C014000400140004401402D
:10C5100030B5026A22F010020262046A426883693E
:10C52000154D2B400D6823F4407343EA052524F094
:10C5300020038C6843EA0413104CA04207D1CC6856
:10C5400023F0800343EA041323F0400305E00C4C7E
:10C55000A04202D00B4CA04207D14C6922F44062A9
:10C5600042EA84028C6942EA840242608561496839
:10C570008163036230BD0000FF8FFFFE002C01408D
:10C58000004001400044014030B5026A22F480724C
:10C590000262046A4268C369144D2B400D6823F09F
:10C5A00003031D4324F400738C6843EA0423104CF6
:10C5B000A04207D1CC6823F4006343EA042323F4A8
:10C5C000806305E00B4CA04202D00B4CA04207D187
:10C5D0004C6922F4405242EA04128C6942EA041285
:10C5E0004260C5614968C163036230BD8FFFFEFFD1
:10C5F000002C0140004001400044014030B5026A77
:10C6000022F480520262046A4268C3690F4D24F426
:10C6100000542B400D6823F4407343EA05238D68D2
:10C6200044EA05340A4DA84205D00A4DA84202D07A
:10C63000094DA84204D14D6922F4804242EA851294
:10C640004260C36149680164046230BDFF8FFFFE30
:10C65000002C0140004001400044014030B5026A16
:10C6600022F480320262046A4268436D0E4D2B4010
:10C670000D681D4324F400330C8943EA04430B4C3A
:10C68000A04205D00A4CA04202D00A4CA04204D1DC
:10C690004C6922F4803242EA0422426045654968CE
:10C6A0008165036230BD00008FFFFEFF002C01405A
:10C6B000004001400044014030B5026A22F480127B
:10C6C0000262046A4268436D0E4D24F400142B404C
:10C6D0000D6843EA05230D8944EA05540A4DA84232
:10C6E00005D00A4DA84202D0094DA84204D14D6997
:10C6F00022F4802242EA8522426043654968C1658E
:10C70000046230BDFF8FFFFE002C0140004001405D
:10C710000044014070B505680024AA6822F0700347
:10C720004A681A431E4B1A400B681343AB604A68B1
:10C7300012F00F0F31D11211082A2ED2DFE802F0C9
:10C740002E2E2E2E0B2127040B69D1E90221006821
:10C75000FFF790FE22E00A68052A10D00268136AEB
:10C76000156A25F00105156202689569096925F0C9
:10C77000F00545EA01119161006803620EE00120B5
:10C7800070BD0A698968006800F00CF806E00A6963
:10C790008968006800F040F800E00124204670BD80
:10C7A000F8FFFEFF10B5036A046A24F00104046276
:10C7B000846924F0F00444EA021423F00A020A43D4
:10C7C0008461026210BD000070B5046A24F00104A7
:10C7D00004628469056A0E4EB04205D0B0F1804F04
:10C7E00002D00C4EB04203D124F00304144301E004
:10C7F00044F001041A0724F0F00444EA126225F020
:10C800000A0301F00A0119438261016270BD000050
:10C81000002C01400040014010B5036A23F01003D2
:10C8200003628369046A23F4704343EA023224F00A
:10C83000A00343EA01118261016210BD30B5046AB0
:10C8400024F0100404628469056A24F4407444EA04
:10C85000022222F470444FF6FF7202EA03322243AE
:10C86000A02425F0A00304EA0111194382610162AA
:10C8700030BD90F82410C90706D001684A68836A61
:10C8800022F400321A434A6090F82410890706D532
:10C8900001684A68C36A22F480321A434A6090F8F9
:10C8A0002410490706D501684A68036B22F48022E8
:10C8B0001A434A6090F82410090706D501684A68AF
:10C8C000436B22F400421A434A6090F82410C906D0
:10C8D00006D501688A68836B22F480521A438A6005
:10C8E00090F82410890606D501688A68C36B22F483
:10C8F00000521A438A6090F82410490611D5016845
:10C900004A68036C22F480121A434A60016CB1F544
:10C91000801F06D101684A68436C22F4C0021A43A2
:10C920004A6090F82410090606D501684A68806CB0
:10C9300022F4002202434A607047F8B500260446FC
:10C94000C0F88060FBF750FF0546206800686FF074
:10C950007E47000708D52B4600224FF400112046E1
:10C96000009700F03FFA60B92068006840070AD5D8
:10C970002B4600224FF480012046009700F032FA47
:10C9800008B10320F8BD2020A067E067266684F880
:10C9900074600020F8BD10B5806A0021A0F85A101C
:10C9A000A0F85210FDF771FC10BD70B5846AA06F3D
:10C9B000E56F216889684FF00006090606D5212831
:10C9C00004D1A4F85260204600F0AEF820688068D8
:10C9D000400606D5222D04D1A4F85A60204600F066
:10C9E0007EF8D4F8800040F01000C4F880002046A3
:10C9F000FDF74BFC70BD10B50146806A09680968F7
:10CA000089062DD40021A0F85A10016851E8002FA2
:10CA100022F4807241E80023002BF6D1016808312E
:10CA200051E8002F22F0010241E80023002BF5D14C
:10CA30000168083151E8002F22F0400241E800234C
:10CA4000002BF5D12021C167016E012908D10268B0
:10CA500052E8001F21F0100142E80013002BF6D12C
:10CA6000016E012902D0FDF79DFE10BDB0F85810EF
:10CA7000FDF7A4FB10BD10B5806A016E012902D03C
:10CA8000FDF7BCFE10BDB0F858104908FDF796FB45
:10CA900010BD10B50146806A09680968890616D478
:10CAA0000021A0F852100168083151E8002F22F04F
:10CAB000800241E80023002BF5D1026852E8001FF4
:10CAC00041F0400142E80013002BF6D110BDFDF704
:10CAD00043FF10BD10B5806AFDF74CFF10BD016823
:10CAE00051E8002F22F4907241E80023002BF6D188
:10CAF0000168083151E8002F22F0010241E80023CB
:10CB0000002BF5D1016E012908D1026852E8001FFF
:10CB100021F0100142E80013002BF6D12021C1675B
:10CB20000021016641667047026852E8001F21F04B
:10CB3000C00142E80013002BF6D120218167704725
:10CB40002DE9F0410446016880682269E3691043D9
:10CB5000626900251A431043714F0A68714B1A40ED
:10CB600002430A6020684168E26821F440511143A1
:10CB700041602168A069B94201D0226A10438A68E5
:10CB800022F4306202438A606749236867488B4217
:10CB90000DD1D0F8880010F0030006D0012847D04E
:10CBA000022843D0032830D144E001212EE060491F
:10CBB0008B420BD1D0F8880010F00C0034D0042840
:10CBC00036D0082832D00C281FD133E059498B4287
:10CBD0000BD1D0F8880010F0300025D0102827D0D5
:10CBE000202823D0302810D124E0BB420DD1D0F82A
:10CBF000880010F4406017D0B0F5806F18D0B0F501
:10CC0000006F13D0B0F5406F14D010214A4A0026AF
:10CC10004FF40040BB422FD171B102290FD004293B
:10CC20000FD0082973D10FE00021EFE70221EDE7D3
:10CC30000421EBE70821E9E7FCF7F6F903E01046E9
:10CC400002E0FCF715FAE8B3626802EB42018142A8
:10CC50005DD8B0EB023F5AD8010E030250081818F5
:10CC600071410023F9F71EFF344AA0F5407191424B
:10CC70004DD82168C8604BE0E3694FF6EF778342F7
:10CC800028D1092943D2DFE801F005080B420D4203
:10CC900042421000FCF7C8F906E0FCF7D7F903E0C0
:10CCA000104602E0FCF7E4F960B14100606801EB76
:10CCB0005001B1FBF0F0A0F11001B94227D84FF6B6
:10CCC000F07100E024E00140C0F34200014320681D
:10CCD000C1601DE009291AD2DFE801F005080B192F
:10CCE0000D1919191000FCF79FF906E0FCF7AEF9D1
:10CCF00003E0104602E0FCF7BBF948B1616800EBC5
:10CD00005100B0FBF1F0A0F11001B94205D90125A5
:10CD100066662846A666BDE8F08180B2A9E70000F5
:10CD200000800040F369FFEF00380140001002402E
:10CD300000440040004800400024F400FFFC0F00C5
:10CD400070B54165A0F8582000250446C0F8805011
:10CD50002220E067206FD8B11F49C162216F1F48B0
:10CD600013460863216F1E484863206F8563666D14
:10CD7000216832462431206FFBF788FA40B1102039
:10CD8000C4F8800004F8745F2020A060012070BD0A
:10CD900084F87450206940B1216851E8000F40F4D4
:10CDA000807041E80002002AF6D12068083050E87F
:10CDB000001F41F0010140E80012002AF5D120686F
:10CDC000083050E8001F41F0400140E80012002AFE
:10CDD000F5D1002070BD0000F7C9000877CA00082F
:10CDE000ABC900082DE9F0479A4617460E4604469F
:10CDF0004FF000094FF02008089D4AE0681C48D019
:10CE0000FBF7F2FCA0EB0A00A8422AD84DB3206839
:10CE1000016849073DD5C069C043000539D4216880
:10CE20004FF400600862206850E8001F21F4D071C0
:10CE300040E80012002AF6D12068083050E8001FB0
:10CE400021F0010140E80012002AF5D1C4F87880F1
:10CE5000C4F87C80C4F8808084F874900320BDE816
:10CE6000F087216851E8000F20F4D07041E80002FB
:10CE7000002AF6D12068083050E8001F21F0010197
:10CE800040E80012002AF5D1C4F87880C4F87C800C
:10CE9000E2E72068C06936EA000004D00020B8420A
:10CEA000ACD00020DBE70120F9E7000070B51F4C93
:10CEB0002068C169C943C9061ED4102101622046F9
:10CEC000FDF77EF91A48006840681A49C0F5967067
:10CED00080B208804FF49675401EA84202D22046C8
:10CEE000FDF760FC2A4614491048FDF731FC206824
:10CEF000016841F0100101602068C169090705D48B
:10CF0000C169490702D4C169890709D508210162AD
:10CF1000216804200862216802200862FFF708F9EE
:10CF2000BDE870400148FDF7B1B900006C18002061
:10CF30007419002044000020041A00202DE9F04755
:10CF400001212E4B0D03642600244FF090494FF42D
:10CF5000FA7C4FF4FA67A3F1140208284CD2DFE8F8
:10CF600000F0040C12192229313C9C7294720122A7
:10CF700040212348FBF733FC28E09972A3F806C050
:10CF80009472BDE8F0879972A3F806C09172D680BA
:10CF9000D17206E09972A3F806C09172D680022081
:10CFA0000EE0D78125E09972A3F806C09172D68071
:10CFB000032005E09972A3F806C09172D680042080
:10CFC000D072EEE79972A3F806C0947229464846DB
:10CFD000BDE8F0470122FBF702BC99720520DE8014
:10CFE000D872C825DD811C739C749172D680D07272
:10CFF000D58114739474C4E79C72C1E7C400002007
:10D000000004004830B5334A3148D16900EB810350
:10D01000491C83ED000A032391FBF3F403FB141175
:10D02000D161D0ED000A2C4AF5EEC00AF1EE10FAFB
:10D0300036D0D0ED010AF5EEC00AF1EE10FA2FD08D
:10D04000D0ED020AF5EEC00AF1EE10FA28D08C1CE1
:10D0500094FBF3F503FB154400EB8404F6EE001A91
:10D0600094ED001A4C1C94FBF3F503FB154300EB05
:10D07000830300EB8100D3ED000A90ED000A10EE6F
:10D08000901A164881420EDA11EE101A81420ADD1A
:10D0900010EE101A814206DD31EE000A20EE210A60
:10D0A00082ED000A30BD30EEC12A0D48B0EEC22A32
:10D0B00012EE101A814207DD30EEC02AB0EEC22A0D
:10D0C00012EE101A8142E7DCC2ED000A30BD00000A
:10D0D0007C1B002078000020100000200000A042EF
:10D0E00000002042FEE700000FB4054B10B503A975
:10D0F000044A029800F02AF910BC5DF814FB000005
:10D1000081DA0008280200200907090E002804DB44
:10D1100000F1E02080F80014704700F00F0000F1EB
:10D12000E02080F8141D704710B52DED028BB0EE95
:10D13000408A18EE100AF9F769FD01EE100A18EEA0
:10D14000100AB7EE000A78EE410A10F0004F4FF0D7
:10D150007F4010EE901A12D0B1F13F4F24BF10EE75
:10D16000901AB0EB410F12D210EE901AB1F17C5F21
:10D170001CDD10EE901AB0EB410F17D314E0B1F1A3
:10D180003F4F07D910EE901AB0EB410F02D331EEAA
:10D19000401A0BE010EE901AB1F17C5F06DB10EE46
:10D1A000901AB0EB410F01D331EE001A18EE100ABD
:10D1B000BDEC028B11EE101A61F31E0000EE100A96
:10D1C00010BD02E008C8121F08C1002AFAD170473A
:10D1D0007047002001E001C1121F002AFBD17047F7
:10D1E0002DE9FF5FDDE90220010DDDF838B00243D3
:10D1F00018D044F61050A1F2FF3141430D140F989E
:10D20000012820D0A5EB0B00401C5FEA000A4FF07C
:10D210000004474EDFF81C91A046504616D5CAF1CF
:10D22000000728E00F98012443A2012808D000211C
:10D2300000980F9BC0E90021C0E9024300F082B8CA
:10D240006FEA0B01F4E7CBF10000DEE7074612E0DE
:10D25000F80707D02246334640464946F9F7A3FD72
:10D26000804689462246334610461946F9F79BFD0B
:10D2700004460E467F10002FEAD1DDE90201BAF123
:10D28000000F42464B4602DAF9F78DFD01E0F9F74F
:10D29000FFFD04460E460022284BF9F781FE03D815
:10D2A0004FF0FF30014607E00022254B2046314673
:10D2B000F9F7CAFCF9F75BFE102409E0002C0ADB41
:10D2C0000A220023F9F7EEFB019B30321A55641E47
:10D2D00050EA0102F2D1641C019AC4F11103144412
:10D2E0000F9A012A03D0012208430DD10AE0084316
:10D2F00004D000204FF0110B0F9080E7A3EB0B053B
:10D300006D1E0DE05B4504DD4FF0000205F10105E7
:10D3100004E003DA4FF00002A5F10105002AECD089
:10D3200000980F99C0E90231C0E9004586E7000086
:10D33000000024400000F03F300000000000F043F7
:10D340000000E03F3FBCBDE8C09F00002DE9FF4F5B
:10D3500095B09B468946064600250FE2252877D1E1
:10D3600000242746F84A0121059400E0044316F8FA
:10D37000013F203B01FA03F01042F7D130782A2810
:10D3800011D06FF02F033078A0F13002092A16D89F
:10D39000059A44F0020402EB820203EB42021044BD
:10D3A000761C0590EFE759F8042B0592002A03DA62
:10D3B000504244F40054059044F00204761C307846
:10D3C0002E2816D116F8010F44F004042A280DD097
:10D3D0006FF02F023078A0F13003092B09D807EB4A
:10D3E000870302EB4303C718761CF3E759F8047B65
:10D3F000761C30786C280FD006DC4C2817D06828B3
:10D400000DD06A2814D104E0742810D07A280FD1E6
:10D410000DE044F400140AE044F4801401E044F404
:10D4200040147278824202D104F58014761C761C76
:10D43000307866280BD013DC582877D009DC002818
:10D4400075D04528F6D04628F4D047281AD19DE15A
:10D4500018E0632835D0642879D0652812D195E189
:10D46000702873D008DC6728F1D069286FD06E2847
:10D470000DD06F2806D1B5E073282CD0752875D053
:10D48000782874D05A46179990476D1C75E1C4F3FB
:10D490000250022809D003280DD0D9F80010042822
:10D4A0000DD00D6009F1040967E1D9F80010EA1701
:10D4B000C1E90052F6E7D9F800100D80F2E70D70CF
:10D4C000F0E719F8041B8DF8001000208DF801001A
:10D4D000EA46012003E059F804AB4FF0FF30610742
:10D4E0004FF0000102D40DE008F101018846B94275
:10D4F0000FDA8045F8DB1AF808100029F4D108E0AB
:10D5000008F1010188468142FADB1AF80810002967
:10D51000F6D105985B46A0EB080721463846179AD6
:10D5200000F097FA284400EB080507E04DE029E1F8
:10D530000DE01AF8010B5A4617999047B8F1010807
:10D54000F7D25B4621463846179A13E142E00A2299
:10D550000092C4F302524FF0000A022A08D059F890
:10D5600004CB032A4FEAEC710AD00DE029E02AE04F
:10D5700009F1070121F00702F2E802C1914609E032
:10D580000FFA8CFC4FEAEC71042A03D14FFA8CFCA1
:10D590004FEAEC71002907DA0A460021DCF1000CA1
:10D5A00061EB02012D2202E0220504D52B228DF829
:10D5B0000420012203E0E20701D02022F7E7904691
:10D5C00059E00A2102E010220DE010214FF0000A7C
:10D5D00000910BE010224FF0000A44F004040827E9
:10D5E000009203E008224FF0000A0092C4F30252B6
:10D5F000022A05D059F804CB0021032A08D009E0FB
:10D6000009F1070121F00702F2E802C1914605E0A5
:10D610001FFA8CFC042A01D10CF0FF0C4FF000081B
:10D62000220728D5702806D0009B83F0100353EA08
:10D630000A0305D00EE040228DF80420012208E004
:10D640005CEA010206D030228DF804208DF8050036
:10D6500002229046009B83F0080353EA0A030AD192
:10D660005CEA010201D1620705D530228DF8042061
:10D670004FF001087F1E582804D034A003900EA854
:10D6800002900DE036A0F9E753466046009AF9F79C
:10D6900009FA84460398825C0298401E0290027048
:10D6A0005CEA0100F0D1029806A9081A00F1200AEC
:10D6B000600702D524F4803400E00127574502DDDD
:10D6C000A7EB0A0000E0002000EB0A01009005989B
:10D6D0004144401A0590E00306D45B462146179A60
:10D6E000059800F0B6F90544002706E001A85A465F
:10D6F000C05D179990476D1C7F1C4745F6DBE00322
:10D700000CD55B462146179A059800F0A2F905440E
:10D7100004E030205A46179990476D1C0099481E26
:10D7200000900029F5DC08E0029802995A4600783A
:10D73000491C0291179990476D1CBAF10001AAF19A
:10D74000010AF1DC65E100000928010030313233C3
:10D75000343536373839616263646566000000002D
:10D760003031323334353637383941424344454617
:10D770000000000000F05BF90544761C30780028BA
:10D780007FF4ECAD19B0284600F04EB9620700D422
:10D79000062709F1070222F0070CFCE80223E14604
:10D7A00003F000485FEA080C02D00FF2702C0DE085
:10D7B0005FEA045C02D50FF2682C07E05FEAC47CE4
:10D7C00002D00FF2602C01E0AFF2700C4FF0FF3886
:10D7D00023F00043CDF850C065280CD006DC452866
:10D7E00009D046281DD047283DD13DE0662818D0F5
:10D7F00067287ED138E00021112F01DB112000E0E5
:10D80000781CCDE9000106A90EA8FFF7E9FCDDE9C7
:10D810000F010E9A03910021009207F1010A049171
:10D820004DE04FF000400097CDE9011006A90EA889
:10D83000FFF7D6FCDDE90F0203920E9B119900223F
:10D84000DDF80CA00093049211B9791C00EB010AD9
:10D85000B7EB0A0004D4C0F1FF3007F1010A0490CD
:10D86000AAEB0700019044E0012F00DA0127002114
:10D87000112F01DD112000E03846CDE9000106A995
:10D880000EA8FFF7ADFCDDE90F010E9A0391002110
:10D8900004910092BA4621070CD40399514500DA4D
:10D8A0008A46BAF1010F05DD009AAAF10101515C27
:10D8B000302908D0B84202DA10F1040F06DA01214B
:10D8C000CDE9011015E0AAF10101E9E7002805DC26
:10D8D000049901440491AAEB000102E0411C514566
:10D8E00000DD8A460499401A401C01904FF0004028
:10D8F0000290200704D40198504501DBCDF8048044
:10D9000000208DF84F0002980DF14F07B0F1004F45
:10D9100025D02B200E9002984FF0020800280CDA38
:10D92000404202902D200E9007E00A210298F9F75C
:10D9300038F93031029007F8011DB8F10001A8F163
:10D940000108F2DC02980028EFD1791E0E980870C9
:10D95000307800F0200040F0450007F8020D12A8D2
:10D96000C01B00F107081498007800B1012000EBFB
:10D970000A01019801EBE07105984144401A401EEC
:10D980000590E00306D45B462146179A059800F0FF
:10D9900060F805441498007818B15A4617999047D2
:10D9A0006D1CE00324D55B462146179A059800F0CC
:10D9B00050F805441CE00498002807DBDDE903016A
:10D9C000884203DD0098405C179901E017993020E8
:10D9D0005A469047049805F10105401C04900198AF
:10D9E000401E019004D12E205A46179990476D1C75
:10D9F000BAF10001AAF1010ADDDC05E017F8010B1C
:10DA00005A46179990476D1CB8F10001A8F101081A
:10DA1000F4DC5B462146179A0598ABE62D00000022
:10DA20002B0000002000000030BCBDE8C08F2DE9B5
:10DA3000F041044600251E461746880404D405E03C
:10DA400039462020B0476D1C641EF9D52846BDE834
:10DA5000F0812DE9F041044600251E469046C8039A
:10DA600001D5302700E02027880404D505E0414691
:10DA70003846B0476D1C641EF9D52846BDE8F081D4
:10DA800013B54FF6FF73012269460248FCF7B8FE52
:10DA900000981CBDF018002070B51A4C44F201012A
:10DAA00022789AB142880D4652BAAA4229D1C18839
:10DAB000E26849BA91420CD0002304222946422050
:10DAC00001F0D0F8BDE8704001F0AAB800230822A8
:10DAD00012E0626821698B1800F1080120221846C3
:10DAE000F9F772FE6068294600F580706060E068B2
:10DAF000401C00231A46E060BDE87040422001F05F
:10DB0000B1B870BD9401002030B5A9B0234C12A863
:10DB1000FCF7FCFF224D214612A8AA68FDF716FC6F
:10DB200012A90EA8FCF7CEFF04221E490EA8F9F791
:10DB300018F850B1A868012101EBD0212046F9F76F
:10DB4000A5FD01F06DF829B030BDFEF715FB3822B8
:10DB500015496846F8F7DAFF0EAC94E80F0001ACFF
:10DB600084E80F00A5208DF8140000983822401C8E
:10DB700000900E480C9069460B48F8F7C7FFFEF777
:10DB8000FBFABFF34F8F0A4801680A4A01F4E061CB
:10DB900011430160BFF34F8F00BFFDE7006800082D
:10DBA00094010020181D0020E01C0020DDCCBBAA41
:10DBB0000CED00E00400FA0570B5C1881E4C49BAAE
:10DBC0004AF6BB25B1F5807F05D0B1F5007F1FD0A7
:10DBD000002306221AE0D0F81710807E09BA21F03F
:10DBE000FF010143A160B1F5BE3F02D9002302222B
:10DBF0000CE01248012606EBD1212061F9F746FD21
:10DC000000206060E06026700346024629460DE071
:10DC10008168C27A09BA21F0FF011143A160084965
:10DC2000C068002308601A464FF48041BDE8704088
:10DC3000422001F017B8000094010020006800089D
:10DC4000181D00201CB5104A01789279914201D02C
:10DC5000FF2914D14178032911D18178402900D0BE
:10DC600069B9C188ADF80010062100F0A6F8ADF83A
:10DC70000400022201A96846F8F773FF08B10020EA
:10DC80001CBD01201CBD0000380200201CB5104A3C
:10DC900001789279914201D0FF2914D14178062967
:10DCA00011D18178402900D069B9C188ADF8001040
:10DCB000062100F082F8ADF80400022201A96846AE
:10DCC000F8F74FFF08B100201CBD01201CBD00006B
:10DCD0003802002010B5134A0178927991420AD196
:10DCE000FF2908D14178422905D18178AA2902D19A
:10DCF000C178BB2901D0002010BD0B49098842180A
:10DD0000491E32F8014C89B200F057F8844207D01E
:10DD1000002305224AF6BB21422000F0A3FFEAE7D8
:10DD2000012010BD380200204400002000B58BB057
:10DD3000142269460E48F9F70BFDBDF810004FF0AC
:10DD40001402A0F52541A5390CD00A4905A8F8F719
:10DD5000DDFE142205A90848F8F7D8FE00F070FF90
:10DD60000BB000BD69460448F8F7D0FEF8E70000A4
:10DD700000F8030828FD000838020020FAF732FEF8
:10DD8000FEF75BFAFDF718FCFDF78EFBFDF716FBBF
:10DD9000FDF730FDFDF7A8FDFDF7C4FDFDF75EFCC6
:10DDA000FDF7BEFCFDF786FCFDF77AFD00F02CF8D0
:10DDB000FDF7B0FB00F03AF8FEE770B504464FF609
:10DDC000FF7000224AF201050DE0A35C58400023D9
:10DDD000C60702D085EA500000E040085B1C082B13
:10DDE000F6DB521C92B28A42EFD370BD10B5EFF34E
:10DDF000058111B16FF0050403E0002408B101F0C2
:10DE0000B5F8204610BD0000EFF3058010B16FF0AB
:10DE1000050070470448016811B14FF0FF307047AA
:10DE20000121016000207047F801002010B5EFF3D8
:10DE3000058010B16FF0050010BD08480168012988
:10DE400002D04FF0FF3010BD054A002182F8141DAA
:10DE50000221016001F0F2F8002010BDF80100205D
:10DE60000BE000E0F8B514464FF00005EFF3058233
:10DE700012BB08B301B3A4B1D4E9023263B1502A92
:10DE80001AD32269C2B1676900FB01F6B74213D306
:10DE9000009501F002FA07E072B9226962B962697D
:10DEA00052B9002201F0D8F9050005D00CB1216863
:10DEB00000E0002101F024F82846F8BD2DE9FF41DB
:10DEC0000B464FF00005EFF30581039549BB40B3C6
:10DED0008027182100244AB3166806B13446966993
:10DEE0001EB13146761E382E02D21679F60703D0BF
:10DEF000002004B0BDE8F081566906B1B708D2F839
:10DF000008C0BCF1000F0DD0D5685C2D18D3126984
:10DF10003AB136B18DE806103A46214601F098FC38
:10DF200003900DE0D6685EB912694AB903AACDE93B
:10DF30000012BAB2214601F05BFC012800D0039523
:10DF40000398D6E70349024809680160704700005A
:10DF5000900100208000002003490248C968016048
:10DF6000704700008801002000000020034902489B
:10DF700009690160704700008C010020000000204A
:10DF80000648054942690A6082694A60C2698A6036
:10DF9000006AC86070470000D01C0020000000200C
:10DFA00038B50546A0211D48F8F7C9FD688869798C
:10DFB0001A4C6A7840BA00292ED07D292CD8184BEB
:10DFC0009B79237062704A00A2700022ADF8002095
:10DFD0006B46E21C00F0BEFD00281DD0BDF800001D
:10DFE000C01C81B22046FFF7E8FEBDF800100122F8
:10DFF0002144C870BDF80010000A21440871BDF822
:10E0000000002021401D85B20648FAF7E8FB2A46A9
:10E0100021460548FCF750FC38BD0000301C0020AC
:10E0200038020020000400486C1800202DE9F05F41
:10E030000546A0217248F8F782FD688895F80180AE
:10E0400047BAA88844F2110245BA6D4CB91A6D4816
:10E050000026DFF8B4914FF0060A4FF0080B4FF09E
:10E06000020E97420FD006DC022F43D0112F65D04D
:10E07000481C07D102E02F29FBD167E0A9F8065020
:10E0800000F0DEFD9FE0691E072933D8A9F808508B
:10E0900000F0D6FD99F80600207084F80180A67083
:10E0A000E7702671657151462046FFF786FEA07124
:10E0B000000AE0715D46012220215448FAF78FFBE7
:10E0C0002A4621465248FCF7F7FB0A20FFF78EFE4E
:10E0D000B9F80800FEF762F84EA42046F8F73AFDBA
:10E0E00082B2642321464A48FCF78AFB00F0AEB8AE
:10E0F00000F0F0BD05804E484C494E4B026825B1FA
:10E10000012D08D0022D0ED05DE0D66300680664B4
:10E110000120187005E0D6630068066483F800E00B
:10E12000012008704FE01E700E709FED430A4349B6
:10E1300081ED000AD6630068066444E000EE105AE0
:10E140003F48B8EE400A80ED020A3CE0A5F5AA413E
:10E15000993902D011392BD035E099F8060020709A
:10E1600084F80180A670E7702671657151462046DB
:10E17000FFF723FEA071000AE0715D460122202115
:10E180002248FAF72CFB2A4621462148FCF794FB4B
:10E190003220FFF72BFEBFF34F8F2A4801682A4A2F
:10E1A00001F4E06111430160BFF34F8F00BFFDE751
:10E1B000FF22A9F80620A9F808E006807046FDF7BE
:10E1C000EDFFFDF7B5FF99F80600207084F8018097
:10E1D000A670E7702671657151462046FFF7EDFD88
:10E1E000A071000AE0715D46012220210748FAF77C
:10E1F000F6FA2A46214600F02EB80548FCF75CBB2B
:10E20000301C002084010020380200200004004857
:10E210006C1800204E6577206261756472617465C8
:10E22000206170706C6965640D0A0000180100209F
:10E23000F81600202401002000000000100000203B
:10E24000881B00200CED00E00400FA0530BCBDE89E
:10E25000C05FFFF74DBF30BCBDE8C05FFFF7CDBF6B
:10E2600010B50446A0211248F8F769FCA08841BA0D
:10E27000B1F5804F0ED06FF4804008180FD0012800
:10E2800012D000230722BDE810404AF6BB214220ED
:10E2900000F0E8BC2046BDE81040FFF78DBC2046EA
:10E2A000BDE81040FFF7F8BBBDE81040FFF72CBCFD
:10E2B000301C00202DE9F041134C0F460546E6685E
:10E2C0002068001D00F01EFD681C07D137B12168D1
:10E2D000BDE8F0410D48091D00F064BD20683544DB
:10E2E000B5424560216805D2A06BBDE8F041091D2B
:10E2F00000F040BD606B091D00F03CFDA06A854246
:10E3000000D2A562BDE8F081A801002018220020FB
:10E310002DE9F041054600F051FD2D4CA068401C50
:10E32000A06020682B4F10B1606930B32BE02560EE
:10E33000A068012827D1002606EB860007EB8000A5
:10E3400000F00AFD761C382EF6D3234800F004FDB9
:10E350002148143000F000FD1F48283000F0FCFC7C
:10E360001D483C3000F0F8FC1B48503000F0F4FC35
:10E37000194860631430A06305E02068E96AC06A48
:10E38000884200D82560606A401C60626864E86A60
:10E390002169884200D9206100EB800007EB8000F2
:10E3A000291D00F0FFFC00F029FD606900280CD059
:10E3B0002068E96AC06A884207D208494FF0805055
:10E3C0000860BFF34F8FBFF36F8FBDE8F08100008F
:10E3D000A8010020681D0020C821002004ED00E0F5
:10E3E00038B500F0EBFC104C2068C8B90F4800F0BD
:10E3F000B3FC0E48143000F0AFFC0C48E060143061
:10E4000020610A4B0020F03B009003F150021021E4
:10E410000A2000F042FF206010B105A100F070FD5D
:10E42000BDE8384000F0EABCE40100201C230020D5
:10E43000546D72510000000030B4026C0B46002A8B
:10E440000BD0C1681144C1608468A14201D3016846
:10E45000C16030BC1846F8F759BB30BC70472DE995
:10E46000F041856B174604460026026C82B1C7B1A5
:10E47000E068F8F74BFBE168206C091AE16022685C
:10E48000914202D2A168081AE060022F16D017E06C
:10E490002068A8B9A06801F07FFA06460020A060B5
:10E4A0000EE06068F8F732FB216C60680844606039
:10E4B000A168884204D32068606001E005B16D1E48
:10E4C0006D1CA5633046BDE8F08110B5044690F898
:10E4D000590058B101280CD002280FD0502080F3E9
:10E4E0001188BFF34F8FBFF36F8FFEE7206B00F0F3
:10E4F00099FC2046BDE8104000F094BC10BD00001F
:10E500000F4844F62061420705D0C01D0C4A20F098
:10E510000700821A891A0B4A00230144C2E900034A
:10E520000839183A21F0070111604B600B600B1A93
:10E53000C0E9001393604FF0004053605061704792
:10E54000FC29002014020020144E154CA6F29C4712
:10E550004FF08058DFF84C9012E000BF00F02EFC26
:10E56000F068C568281D00F0CDFBA068401EA060C3
:10E570006068401E606000F041FC2846FFF7A5FF80
:10E5800060680028EAD138680128F9D9C9F8008004
:10E59000BFF34F8FBFF36F8FF2E70000042200201C
:10E5A000A801002004ED00E070B51D46049C51B1A7
:10E5B000C4F80020C4E90F010121204600F0A0FEAC
:10E5C00084F84C5070BD2460F4E700002DE9F05F42
:10E5D0008846DDE90B941546834691009A460A9ECB
:10E5E000A522206BF8F7A4FA6FF00301206B01EB72
:10E5F0008501084420F00707780707D0502080F3F2
:10E600001188BFF34F8FBFF36F8FFEE70025B8F17E
:10E61000000F0FD05FF00000221818F8001082F8E9
:10E62000341018F8001011B1401C1028F4D384F8ED
:10E63000435001E084F83450382E00D33726E66288
:10E64000C4E91365201D00F092FB04F1180000F0EE
:10E650008EFB2461C6F138006462A061656584F8B0
:10E66000585052465946384600F05EFA2060B9F1DB
:10E67000000F01D0C9F8004000F000B830BCBDE880
:10E68000C09F000030B5114900E011460A6882427F
:10E69000FBD34B685C18844203D14068184448603F
:10E6A000084643681C18944209D1084C183C246859
:10E6B000A24209D052681A4442600A681268026095
:10E6C000814200D0086030BD0460F9E714020020E8
:10E6D00070B5002441600B4D0061914206D8D11AFB
:10E6E0008269914206D2011D286907E09A4203D24D
:10E6F000994201D3012403E0011DE86800F03AFBD0
:10E70000204670BDE401002010B5044600F056FB21
:10E71000A06B28B15FF0000400F070FB204610BD34
:10E720000124F9E730B589B03C4D6EE0049800282B
:10E7300006DADDE90601059A90470498002864DBB3
:10E74000069C606910B1201D00F0DCFA03A800F0FF
:10E75000D7F8024604980A2857D2DFE800F00505EA
:10E76000052D334A05052D3394F8280040F00100AB
:10E7700084F828000599A069059B01442046FFF70D
:10E78000A7FF68B3216A2046884794F8280040070D
:10E790003BD5002000900598A16900234218194636
:10E7A000204601F003FAD8B9502080F31188BFF356
:10E7B0004F8FBFF36F8FFEE714F8280F20F0010092
:10E7C000207022E094F8280040F0010084F828002E
:10E7D0000598A06128B1811813462046FFF778FFFD
:10E7E00013E0502080F31188BFF34F8FBFF36F8F7A
:10E7F000FEE794F82800810703D4204600F012FBBE
:10E8000003E020F0010084F82800002204A9286811
:10E8100000F0CAFE002889D109B030BDE401002013
:10E820002DE9FC410F46054600F04CFC01A800F024
:10E8300067F80446019818B101F026F9BDE8FC819B
:10E84000254EAFB130690068D0B30027291B3A4686
:10E85000306800F069FB01F017F90028EED11F497C
:10E860004FF080500860BFF34F8FBFF36F8FE5E725
:10E87000A542EBD801F008F9F0682746C068C468E3
:10E88000201D00F03FFA94F82800410719D5A0692F
:10E890002B4641193A462046FFF71AFFA8B100203F
:10E8A0000346014600902A46204601F07FF960B9F0
:10E8B000502080F31188BFF34F8FBFF36F8FFEE7B7
:10E8C00007E020F0010084F82800216A20468847EC
:10E8D000B4E70127BAE70000E401002004ED00E0FE
:10E8E0000648416B096829B1416BC968C968496824
:10E8F000816270474FF0FF31FAE70000A801002065
:10E9000070B5054600F0DEFF064E0446B06884424E
:10E9100003D200F009F8012000E000202860204622
:10E92000B46070BDE4010020F8B5194D20E0C06866
:10E93000C4680668201D00F0E5F9216A2046884772
:10E9400094F82800400713D5A0693044B04206D996
:10E9500024616060211DE86800F00CFA08E00020E6
:10E960000346014600903246204601F01FF938B1B7
:10E97000E86801680029DAD12969C5E90310F8BD02
:10E98000502080F31188BFF34F8FBFF36F8FFEE7E6
:10E99000E401002008484068401C4FF0500080F31C
:10E9A000118804D0BFF34F8FBFF36F8FFEE7BFF323
:10E9B0004F8FBFF36F8FFEE71C020020074CE0680B
:10E9C000016841B1C0680021D0F80000FFF728FFBE
:10E9D000FFF7A8FEF3E701210020F7E7E40100209C
:10E9E0002DE9F041044600F0E9F994F9455004F1AD
:10E9F000240609E0606A48B1304601F00DF808B11C
:10EA000000F0E2FA6D1E6DB2002DF3DC4FF0FF3620
:10EA100084F8456000F0F2F900F0D0F994F9445020
:10EA200004F1100709E0206948B1384600F0F4FF0E
:10EA300008B100F0C9FA6D1E6DB2002DF3DC84F848
:10EA40004460BDE8F04100F0D9B900002DE9F04183
:10EA50000546002700F036FB324E306808B9FFF754
:10EA60004FFD706905424ED1C5B3083568070ED019
:10EA700005F00700C0F108000544680707D05020E2
:10EA800080F31188BFF34F8FBFF36F8FFEE72DB375
:10EA90007068854237D82348183001460C6801E079
:10EAA00020460C466168A94202D221680029F7D1AC
:10EAB00031688C4227D00768216801606068083798
:10EAC000411B10290FD96019420708D0502080F34C
:10EAD0001188BFF34F8FBFF36F8FFEE713E04160E4
:10EAE0006560FFF7CFFD61687068401A7060B268BA
:10EAF000904200D2B060706901430020C4E9000177
:10EB0000F068401CF06000F0BFFF780707D050208D
:10EB100080F31188BFF34F8FBFF36F8FFEE7384646
:10EB2000BDE8F081FC01002010B5031F4FF0807498
:10EB30001C601B1F21F001011960191F044B0B60A1
:10EB400014390A60091F6FF0020244380A6010BDD0
:10EB500095E900082DE9F0479A460023DFF8BC90BC
:10EB60004FE000254FEA090606EBC50736F83540A9
:10EB7000BF78A0422744BFB24AD3B84248D2041B50
:10EB80001FFA84FC3C1AA4B2A14200D20C4609EB45
:10EB9000C5056F68ED7875B300251AE00CEB050626
:10EBA000B6B24FEA560846F3000657F82880761C9E
:10EBB00002D04FEA184601E01FFA88F64FEA1628FD
:10EBC00002F803805B1C9BB2D6545B1C6D1C9BB28D
:10EBD000ADB2A542E2D310E00CEB050637F81660A3
:10EBE0004FEA162802F803805B1C9BB2D6545B1CCC
:10EBF0006D1C9BB2ADB2A542EED32044091B80B27E
:10EC000089B20029ADD1AAF800300120BDE8F08713
:10EC10006D1C0B2DA8D30020F8E700002801002070
:10EC200070B5054C0025102165600448A560F7F714
:10EC300086FFE560257070BD94010020181D00203E
:10EC400010B5064C01212046F8F720FD2046BDE80E
:10EC5000104005220249F8F78FBD000000F80308B4
:10EC60003802002010B5184C88B0A4798DF8004007
:10EC70008DF80100080A8DF8020041208DF804008B
:10EC800000208DF805008DF806208DF80700180A81
:10EC90008DF808008DF803108DF809300A216846B8
:10ECA000FFF78BF88DF80A00000A8DF80B000C2492
:10ECB000012220210548F9F792FD224669460448C1
:10ECC000FBF7FAFD08B010BD380200200004004830
:10ECD0006C18002010B54FF4967421460748F7F7DA
:10ECE0002EFF07480068016841F0100101602246CC
:10ECF000BDE8104001490248FBF72ABD041A002074
:10ED00006C180020D0E9013201699A60D0E9012332
:10ED10005A604A68824201D182684A6000220261D8
:10ED20000868401E0860086870470000034B0360D5
:10ED300003F15C00086080201060704744230020CD
:10ED4000044B036003F15C0008604FF480701060B6
:10ED500070470000A025002000F108014FF0FF32AD
:10ED6000C0E90112C160016100210160704700210A
:10ED70000161704730B50B685A1C02D000F10802DF
:10ED800002E0026904E02246546825689D42FAD9EF
:10ED900053684B6099608A60516008610168491C42
:10EDA000016030BD42684A6093688B609368596027
:10EDB000916008610168491C01607047502080F330
:10EDC0001188BFF34F8FBFF36F8F0A494868401C0B
:10EDD000486001280CD10848006810F0FF0F07D0E8
:10EDE000502080F31188BFF34F8FBFF36F8FFEE782
:10EDF000704700001C02002004ED00E0084948684C
:10EE000028B1401E486001D180F31188704750201E
:10EE100080F31188BFF34F8FBFF36F8FFEE70000C1
:10EE20001C02002070B500282AD0164DA0F108045D
:10EE300060686969084207D1502080F31188BFF3E8
:10EE40004F8FBFF36F8FFEE722683AB1502080F3F7
:10EE50001188BFF34F8FBFF36F8FFEE78843606069
:10EE600000F030F960686968084468602046FFF780
:10EE700009FC2869401C2861BDE8704000F004BE10
:10EE800070BD0000FC0100204FF0E0200021016176
:10EE9000816105494FF47A720968B1FBF2F1491EAC
:10EEA00041610721016170477400002010B5F7F738
:10EEB000D3FD114910280ED300F1E02090F8F003A3
:10EEC0000A78904207D2502080F31188BFF34F8F09
:10EED000BFF36F8FFEE709480068896800F4E060BF
:10EEE000884207D9502080F31188BFF34F8FBFF3BA
:10EEF0006F8FFEE710BD00001C0200200CED00E04B
:10EF000010B5084B002200BF53F832401CB1521C10
:10EF1000082AF9D310BD43F8321003EBC201486050
:10EF200010BD0000281D002070B515460E46044691
:10EF3000FFF744FF94F944100020491C01D184F8E4
:10EF4000440094F94510491C01D184F84500FFF7AD
:10EF500055FFA06B28B92A46314604F1240000F081
:10EF600051F82046BDE87040FFF73ABD10B50200E9
:10EF700014D00F48006B38B1502080F31188BFF3D4
:10EF80004F8FBFF36F8FFEE700F09CF80021104613
:10EF9000FFF790F900F078FD002807D105494FF000
:10EFA00080500860BFF34F8FBFF36F8F10BD00001C
:10EFB000A801002004ED00E002490A6A0260C96865
:10EFC00041607047A801002001490120C8617047D5
:10EFD000A801002010B50C4650B109490968183144
:10EFE000FFF7C8FE2046BDE810400121FFF762B9D7
:10EFF000502080F31188BFF34F8FBFF36F8FFEE770
:10F00000A801002070B514460D4668B10A49096888
:10F010001831FFF7C7FE0CB14FF0FF3521462846E7
:10F02000BDE87040FFF746B9502080F31188BFF368
:10F030004F8FBFF36F8FFEE7A801002030B587B078
:10F040000024039405AA04A903A80494FFF76EFE04
:10F05000DDE903010094CDE90110002315A1174853
:10F06000059A00F0F5FB164D0028E8621FD000F06D
:10F070006DFD012809D0401C19D1502080F3118862
:10F08000BFF34F8FBFF36F8FFEE7502080F31188DF
:10F09000BFF34F8FBFF36F8F4FF0FF30A862012097
:10F0A0006861EC6007B0BDE8304000F045B807B0DB
:10F0B00030BD000049444C450000000049E500080F
:10F0C000A80100200248016B491C01637047000041
:10F0D000A8010020164810B5016B11B10121C161D2
:10F0E00010BD0021C1610169124A01E0B9B1491E98
:10F0F00001EB810352F82330002BF7D001EB8103A1
:10F1000002EB830202F1080453685B685360A34278
:10F1100001D15B685360DA680260016110BD502064
:10F1200080F31188BFF34F8FBFF36F8FFEE70000AE
:10F13000A8010020681D00201CB537480168374A27
:10F14000914207D1502080F31188BFF34F8FBFF356
:10F150006F8FFEE700683149491E884207D1502071
:10F1600080F31188BFF34F8FBFF36F8FFEE72C49F9
:10F1700008780190FF20087008788DF800009DF84D
:10F1800000009DF8002000F0F000904207D05020D1
:10F1900080F31188BFF34F8FBFF36F8FFEE79DF8A9
:10F1A0000000204C00F0500020700720A06005E017
:10F1B0009DF8002052008DF80020401E9DF8002090
:10F1C0001206F5D4A060032807D0502080F31188E0
:10F1D000BFF34F8FBFF36F8FFEE74FF44070A06017
:10F1E000019808700C482030016841F470010160FA
:10F1F000016841F070410160FFF746FE0020606049
:10F20000F7F7F2FB0848016841F040410160F7F769
:10F21000D7FB00201CBD000000ED00E071C20F41D3
:10F2200000E400E01C02002034EF00E010B55020A4
:10F2300080F31188BFF34F8FBFF36F8F00F048FB4F
:10F2400018B104494FF080500860002080F3118805
:10F2500010BD000004ED00E0F8B517460E460500AD
:10F2600013D005FB06F05030FFF7F0FB04000AD086
:10F27000002084F8460004F150023B4631462846FF
:10F280000094FFF791F92046F8BD502080F31188D3
:10F29000BFF34F8FBFF36F8FFEE738B5049D18B1F2
:10F2A00053B1CAB181B120E0502080F31188BFF37F
:10F2B0004F8FBFF36F8FFEE7502080F31188BFF3AD
:10F2C0004F8FBFF36F8FFEE7502080F31188BFF39D
:10F2D0004F8FBFF36F8FFEE739B1502080F3118855
:10F2E000BFF34F8FBFF36F8FFEE750241C460123FF
:10F2F00084F846302B460094FFF756F9204638BD77
:10F3000070B50D46040025D0FFF758FDD4E90F2055
:10F31000216802FB0011A1600021A16321686160E6
:10F320000A46D4E90F01401E00FB0121E16021469D
:10F330004FF0FF3001F8440F487004F110008DB118
:10F34000FFF70AFD04F12400FFF706FDFFF756FD65
:10F35000012070BD502080F31188BFF34F8FBFF3A1
:10F360006F8FFEE721690029F0D000F055FB0028DF
:10F37000ECD004494FF080500860BFF34F8FBFF3CB
:10F380006F8FE3E704ED00E02DE9FF4782B01D46F3
:10F390008A464FF00008040003D0BAF1000F08D0ED
:10F3A00011E0502080F31188BFF34F8FBFF36F8FB0
:10F3B000FEE7206C38B1502080F31188BFF34F8FE7
:10F3C000BFF36F8FFEE7022D0AD1E06B012807D053
:10F3D000502080F31188BFF34F8FBFF36F8FFEE78C
:10F3E00000F062FA3F4F4FF000094FF0805648B9E5
:10F3F000049838B1502080F31188BFF34F8FBFF3CA
:10F400006F8FFEE7FFF7DAFCA06BE16B884207D352
:10F41000022D05D00498D0B1B8F1000F1AD01EE02B
:10F420002A4651462046FFF71AF8616A19B104F1DD
:10F43000240000F0F1FA20B13E60BFF34F8FBFF31C
:10F440006F8FFFF7DBFC012006B0BDE8F087FFF708
:10F45000D5FC22E06846FFF7AFFD4FF00108FFF74B
:10F46000CDFCFFF72FFEFFF7A9FC94F94400401CE8
:10F4700001D184F8449094F94500401C01D184F8EE
:10F480004590FFF7BBFC04A9684600F077F930B15E
:10F490002046FFF7A5FA00F0F7FA0020D4E7FFF7BF
:10F4A0008DFCA06BE16B884213D1FFF7A7FC04F140
:10F4B00010000499FFF78EFD2046FFF791FA00F047
:10F4C000E3FA00289ED13E60BFF34F8FBFF36F8FEA
:10F4D00098E7FFF793FC2046FFF782FA00F0D4FA92
:10F4E00090E7000004ED00E02DE9F0471F4690464C
:10F4F0008946040003D0B9F1000F08D011E0502074
:10F5000080F31188BFF34F8FBFF36F8FFEE7206C3E
:10F5100038B1502080F31188BFF34F8FBFF36F8F46
:10F52000FEE7022F0AD1E06B012807D0502080F3BC
:10F530001188BFF34F8FBFF36F8FFEE7FFF7B6FC65
:10F540005020EFF3118680F31188BFF34F8FBFF384
:10F550006F8FA06BE16B884206D3022F04D000208E
:10F5600086F31188BDE8F08794F94550A06B3A46C0
:10F5700049462046FEF773FF681C04D06D1C84F8D2
:10F5800045500120ECE7606A0028FAD004F124001D
:10F5900000F042FA0028F4D0B8F1000FF1D00121B8
:10F5A000C8F80010EDE700002DE9F747002683B00A
:10F5B0008A46040003D0BAF1000F08D011E05020B1
:10F5C00080F31188BFF34F8FBFF36F8FFEE7206C7E
:10F5D00038B1502080F31188BFF34F8FBFF36F8F86
:10F5E000FEE700F061F9DFF8F4804FF000094FF01A
:10F5F000805748B9059838B1502080F31188BFF37F
:10F600004F8FBFF36F8FFEE7FFF7D8FBA56BC5B138
:10F6100051462046FEF710FF6D1EA563206950B1CC
:10F6200004F1100000F0F8F928B1C8F80070BFF339
:10F630004F8FBFF36F8FFFF7E1FB012006B0BDE8EE
:10F64000F087059808B11EB106E0FFF7D7FB27E069
:10F650006846FFF7B1FC0126FFF7D0FBFFF732FD4C
:10F66000FFF7ACFB94F94400401C01D184F84490AE
:10F6700094F94500401C01D184F84590FFF7BEFB8A
:10F6800005A9684600F07AF8002820460AD0FFF75E
:10F69000A7F900F0F9F92046FFF736F80028B3D0B3
:10F6A0000020CBE7FFF730F890B104F12400059972
:10F6B000FFF790FC2046FFF793F900F0E5F90028EA
:10F6C000A2D1C8F80070BFF34F8FBFF36F8F9BE7D5
:10F6D0002046FFF785F900F0D7F995E704ED00E043
:10F6E0002DE9F04790468946040003D0B9F1000F98
:10F6F00008D011E0502080F31188BFF34F8FBFF383
:10F700006F8FFEE7206C38B1502080F31188BFF373
:10F710004F8FBFF36F8FFEE7FFF7C8FB5020EFF36B
:10F72000118680F31188BFF34F8FBFF36F8FA76BE4
:10F73000F7B194F9445049462046FEF77DFE7F1EFE
:10F74000A763681C04D06D1C84F84450012010E0AD
:10F7500020690028FAD004F1100000F05DF90028BB
:10F76000F4D0B8F1000FF1D00121C8F80010EDE796
:10F77000002086F31188BDE8F08700002DE9F041F4
:10F780000C46050011D0C4B1FFF718FB174BDA681F
:10F790006E682068911B471C17D02F681B6A9F4218
:10F7A00019D0964217D8012410E0502080F3118818
:10F7B000BFF34F8FBFF36F8FFEE7502080F31188A8
:10F7C000BFF34F8FBFF36F8FFEE70024FFF716FBE9
:10F7D0002046BDE8F081884205D9401A20602846BD
:10F7E000FFF7EAFBF1E700202060DCE7A80100203A
:10F7F0002DE9FF5F8346DDE90E87994616468A4666
:10F800009000FFF723F905001CD05C20FFF71EF9DC
:10F81000040014D00020256384F85900CDE902408B
:10F82000CDE900874B46324651465846FEF7CEFE9C
:10F830002046FEF76DFD012004B000F006B8284612
:10F84000FFF7F0FA4FF0FF30F6E730BCBDE8C09F9D
:10F85000F0B585B0DDE90B640A9DA6B1DCB15C278B
:10F8600000972663022684F85960002604AFCDE98C
:10F870000246CDE90057FEF7A9FE2046FEF748FDF7
:10F88000049805B0F0BD502080F31188BFF34F8F6E
:10F89000BFF36F8FFEE7502080F31188BFF34F8FC7
:10F8A000BFF36F8FFEE700000548416919B1006B97
:10F8B00018B10020704701207047022070470000F7
:10F8C000A80100200148C06870470000A80100207E
:10F8D0002DE9F0412E4C0027206B28B1A069401C77
:10F8E000A0613846BDE8F081E668761CE66013D179
:10F8F000606B006838B1502080F31188BFF34F8FE0
:10F90000BFF36F8FFEE7606BA16B6163A063206A3A
:10F91000401C2062FEF7E4FFA06ADFF87880864290
:10F9200009D3606B0068A0B1606BC068C568686887
:10F93000864211D2A0622068C06A00EB800158F8AC
:10F940002100012800D90127E0690028C9D001273A
:10F95000C7E74FF0FF30EDE7281DFFF7D3F9A86A9E
:10F9600018B105F11800FFF7CDF9E86A216988425E
:10F9700000D9206100EB800108EB8100291DFFF711
:10F9800011FAE86A2168C96A8842CAD30127C8E720
:10F99000A8010020681D002070B504004FF0000190
:10F9A00033D01B4D2868844207D0502080F3118843
:10F9B000BFF34F8FBFF36F8FFEE7206D38B1401E4E
:10F9C0002065E36CE26A9A421FD040B11DE05020EE
:10F9D00080F31188BFF34F8FBFF36F8FFEE7201DB9
:10F9E000FFF790F9E06CE062C0F13800A061E06AD6
:10F9F0002969884200D92861064900EB800001EBA3
:10FA00008000211DFFF7CEF90121084670BD0000DE
:10FA1000A8010020681D002070B5C068C46854B1FA
:10FA200004F118000646FFF76DF9144D286B50B12C
:10FA30003146134815E0502080F31188BFF34F8FF3
:10FA4000BFF36F8FFEE7201DFFF75CF9E06A2969BD
:10FA5000884200D928610B4900EB800001EB80004F
:10FA6000211DFFF79FF9E06A2968C96A884202D917
:10FA70000120E86170BD002070BD0000A8010020D9
:10FA8000F0210020681D00202DE9F0472C4D0024B6
:10FA90002746286B38B1FFF791F9286B401E286381
:10FAA000286B40B146E0502080F31188BFF34F8FA0
:10FAB000BFF36F8FFEE7A968224E0120D1B3A6F5F0
:10FAC000916980463068E0B1F068C46804F11800BC
:10FAD000FFF718F9201DFFF715F9E06A2969884238
:10FAE00000D9286100EB800109EB8100211DFFF79F
:10FAF00059F9E06A2968C96A8842E3D3C5F81C80CD
:10FB0000E0E70CB1FEF7ECFEAC694CB14FEA080639
:10FB1000FFF7DEFE00B1EE61641EF9D10020A8619E
:10FB2000E86938B10849012738070860BFF34F8FEB
:10FB3000BFF36F8FFFF762F93846BDE8F08700002A
:10FB4000A8010020F021002004ED00E010B586B0EF
:10FB5000FEF746FC114C2068B8B1002003900490D9
:10FB600005AA04A903A8FFF7EBF8DDE903210220A9
:10FB70008DE8070000230AA10B48059AFFF768FEED
:10FB8000606010B106B0012010BD502080F31188D4
:10FB9000BFF34F8FBFF36F8FFEE70000E40100203B
:10FBA000546D722053766300BDE900082DE9FF41D2
:10FBB0001E46134602000A9D4FF0000016D0144C5A
:10FBC0002768002F0FD0CDE900130292062917DA1B
:10FBD000FFF76AFE02284FF000030FD000226946AB
:10FBE0002068FFF7D1FB04B0BDE8F081502080F31E
:10FBF0001188BFF34F8FBFF36F8FFEE72A46EEE702
:10FC00000023324669463846FFF76EFCEBE70000FA
:10FC1000E4010020BCFD000800000000000000001E
:10FC200000000000000000000002000030000000A2
:10FC300000000000000000008CFD00080000000033
:10FC400000000000000000000000000000020000B2
:10FC500018000000000000000000000098FD0008EF
:10FC60000000000000000000000000000000000094
:10FC70000008000018000000000000000000000064
:10FC8000A4FD0008000000000000000000000000CB
:10FC90000000000000020000100000000000000052
:10FCA00000000000B0FD000800000000000000009F
:10FCB0000000000000000000000400001800000028
:10FCC00000000000000000007CFD000800000000B3
:10FCD0005C150020500000009C020020C0120000B3
:10FCE00000000000000000000102030406070809EC
:10FCF000A0860100400D0300801A060000350C00AC
:10FD000040420F0080841E0000093D0000127A006E
:10FD10000024F40000366E010048E801006CDC02AB
:10FD200000000000010203044FB907000000FF00BB
:10FD30000200FF000619010AA5A5000080000000CE
:10FD400000000000000000000000000000000000B3
:10FD500000000000000000000000000000000000A3
:10FD60000000000000000000000000000000000093
:10FD700000000000000000000000000075617274C7
:10FD80003438357278717565756500005265616447
:10FD90005461736B000000004465616C5461736BC7
:10FDA00000000000436F6D6D6F6E5461736B000057
:10FDB0004D6F746F725461736B000000486967681F
:10FDC0006573745461736B00E8FD00080000002047
:10FDD0002C0200004071000860FE00082C02002088
:10FDE000F4790000D2D10008014832010A19101C30
:10FDF000D10B33093D6071FA486912040310484081
:10FE00001914DA801CE204694812480A130820E138
:10FE100016400201380215200240011380011B2008
:10FE200010081A3E101A11081A4008142040031A2C
:10FE300042081A01AA1A82201A02081A8408120318
:10FE40001C020188081A05081A8C081A07081A905B
:10FE5000081209150801D01C02A0201AAA0181006D
:040000050800698DF9
:00000001FF
